:020000040800F2
:10000000480F002439030008B74D0090C319009031
:1000100045030008030300904B58009000000000C7
:10002000000000000000000000000000FD500090F3
:100030000503009000000000B94D0090FF500090B3
:100040005303000853030008530300085303000838
:100050005303000853030008530300085303000828
:100060005303000853030008530300085303000818
:100070005303000853030008530300085303000808
:1000800053030008530300085303000853030008F8
:1000900053030008530300085303000853030008E8
:1000A00053030008530300085303000853030008D8
:1000B00053030008530300085303000853030008C8
:1000C00053030008530300085303000853030008B8
:1000D0005303000851150008530300085303000898
:1000E00053030008530300080000000053030008F6
:1000F0005303000853030008530300085303000888
:100100005303000853030008530300085303000877
:100110005303000853030008530300085303000867
:100120005303000853030008530300085303000857
:100130005303000853030008530300085303000847
:1001400000000000000000000000000000000000AF
:100150005303000853030008530300085303000827
:100160005303000853030008530300085303000817
:100170005303000853030008530300085303000807
:1001800053030008530300085303000853030008F7
:1001900053030008530300085303000853030008E7
:1001A00053030008530300085303000853030008D7
:1001B00053030008530300085303000853030008C7
:1001C00053030008530300085303000853030008B7
:1001D00053030008530300085303000853030008A7
:1001E0005303000853030008530300085303000897
:1001F0005303000853030008530300085303000887
:100200005303000853030008530300085303000876
:100210005303000853030008530300085303000866
:1002200053030008530300085303000800000000B4
:1002300053030008530300080000000053030008A4
:100240005303000853030008530300085303000836
:100250005303000853030008530300085303000826
:100260005303000853030008530300085303000816
:100270005303000853030008530300080000000064
:1002800053030008000000005303000800000000B2
:10029000000000005303000800F002F800F03CF8F2
:1002A0000AA090E8000C82448344AAF10107DA45D1
:1002B00001D100F031F8AFF2090EBAE80F0013F0E7
:1002C000010F18BFFB1A43F001031847B4150000D3
:1002D000D4150000103A24BF78C878C1FAD8520764
:1002E00024BF30C830C144BF04680C6070470000B0
:1002F0000023002400250026103A28BF78C1FBD82F
:10030000520728BF30C148BF0B6070471FB501F0CE
:10031000A9FA1FBD10B510BD00F0AAF81146FFF7ED
:10032000F5FF01F085F900F0C8F803B4FFF7F2FF1C
:1003300003BC01F03FF90000094880470948004725
:10034000FEE7FEE7FEE7FEE7FEE7FEE7FEE7FEE785
:10035000FEE7FEE704480549054A064B70470000E2
:10036000CD1400089902000848030024480F002417
:100370004805002448050024704753EA020C00F0A9
:1003800069802DE9F04B4FF00006002B1FBFB3FA38
:1003900083F503FA05F424FA05F65E4012BF16430E
:1003A000B2FA82F502FA05F4C5F120051EBF22FA61
:1003B00005FC44EA0C04203556EA044C4FEA144488
:1003C00018BF641C4FF000084FF00009904271EB19
:1003D000030C39D3002919BFB1FA81F701FA07F6E6
:1003E000B0FA80F700FA07F6C7F120071EBF20FA1F
:1003F00007FC46EA0C062037B6FBF4FCA7EB050722
:10040000103F07F01F0BCBF120060CFA0BFB2CFA68
:1004100006F644BFB3460026202FA4BF5E464FF029
:10042000000B5BEA060C08BF4FF0010B19EB0B0940
:10043000ABFB027C48EB0608C01B06FB02CC0BFBA7
:1004400003CC71EB0C01C1E70B460246414648461E
:10045000BDE8F08B13B54FF000004FF00001AFF393
:100460000080BDE81C407047704770477047704778
:10047000754600F02BF8AE4605006946534620F05D
:100480000700854618B020B5FFF764FFBDE820409F
:100490004FF000064FF000074FF000084FF0000B40
:1004A00021F00701AC46ACE8C009ACE8C009ACE8F3
:1004B000C009ACE8C0098D46704710B50446AFF3DB
:1004C00000802046BDE81040FFF72FBF004870476E
:1004D000E402002440F6650CC9F2000C604741F2CA
:1004E000317CC9F2000C604741F2257CC9F2000C56
:1004F000604741F61B1CC9F2000C604744F2716C66
:10050000C9F2000C604741F6C51CC9F2000C6047F7
:1005100045F21D0CC9F2000C604741F6555CC9F26A
:10052000000C604744F2C75CC9F2000C604744F617
:10053000D57CC9F2000C604741F6452CC9F2000C8D
:10054000604744F69D7CC9F2000C604744F2515C60
:10055000C9F2000C604744F6B17CC9F2000C604758
:1005600041F6B10CC9F2000C60470000F0B5BFF3D2
:100570004F8FBFF36F8F1D4900200860BFF34F8F6F
:10058000BFF36F8F1A4C216841F400312160BFF333
:100590004F8FBFF36F8F164970310860BFF34F8FD5
:1005A000081F006843F6FF75104E1036C0F34E3139
:1005B000C0F3C90305EA4112184642EA8077376062
:1005C000401EFAD2491EF5D2BFF34F8F206840F487
:1005D00080302060BFF34F8FBFF36F8F03484C30E4
:1005E000016841F004010160F0BD000050EF00E03F
:1005F00014ED00E00248016841F00101016070471C
:10060000200400582DE9F84F6C4C00224FF0B04AFE
:100610004FF0010B4FF0030E4FF00F090B680BFA70
:1006200002F73B40BB4270D14D68022D01D0122D24
:1006300012D1D50800EB850CDCF820605507ED0ED3
:1006400009FA05F826EA0806D1F8108008FA05F834
:1006500048EA0608CCF82080D0F80080560091F8CF
:1006600004C00EFA06F50CF0030C28EA05080CFA93
:1006700006FC4CEA080CC0F800C0D1F804C0BCF17C
:10068000010F08D0BCF1020F05D0BCF1110F02D050
:10069000BCF1120F16D1D0F808C0D1F80C802CEAAA
:1006A000050C08FA06F848EA0C08C0F80880D0F8EB
:1006B00004C02CEA070C0F79C7F30017974047EAEC
:1006C0000C074760C768AF438D68B5403D43C560C0
:1006D0004D68ED006BD53A4D2E6846F002062E604F
:1006E0002D6822F0030606F1B04605F002050095DC
:1006F000D6F808C495072F0F09FA07F52CEA050C60
:10070000304DA84202D100252EE050E02E4DA842E7
:1007100001D1012528E02D4DA84201D1022523E079
:100720002B4DA84201D103251EE02A4DA84201D13C
:10073000042519E0284DA84201D1052514E0274DD4
:10074000A84201D106250FE0254DA84201D1072579
:100750000AE0244DA84201D1082505E0224DA84217
:1007600001D1092500E00A25BD4045EA0C05C6F87F
:10077000085425684E689D43F60300D51D43256047
:1007800065684E689D43B60300D51D436560DAF881
:10079000005056464F689D43FF0200D51D4335600B
:1007A00075684F689D43BF0200D51D437560521C9C
:1007B000102AFFF433AFBDE8F88F00008000005826
:1007C000F44402580000025800040258000802587D
:1007D000000C025800100258001402580018025869
:1007E000001C0258002002580024025800690840EA
:1007F00000D00120704742694A40426170470AB107
:10080000018370474183704701488068704700004A
:100810001400002402488168027811448160704706
:1008200014000024032010B500F0A2F80F2000F0FF
:1008300007F808B1012010BD00F06CF8002010BDD1
:1008400070B50D4D04464FF47A712878B1FBF0F085
:100850000A490968B1FBF0F000F0A4FC48B9102C7B
:1008600007D200222146501E00F062F800206C6082
:1008700070BD012070BD00001400002400000024A1
:10088000134A41781160111D03780A1DE3B14368D2
:100890000B60017BC37A090741EA0361837A41EA6D
:1008A000C341437B41EA8341837B41EA4341C37BAC
:1008B00041EA0341437A41EA0321037A007841EA9D
:1008C00043010143116070470020086010607047C9
:1008D00098ED00E0BFF35F8F0448016821F4803198
:1008E00001600249002070310860704724ED00E08B
:1008F000074940F00100086005487038016841F47C
:1009000080310160BFF34F8FBFF36F8F70470000DE
:1009100094ED00E07047002809DB012100F01F0280
:1009200091404009800000F1E020C0F800117047BC
:100930000E4BF0B41B68C3F30223C3F10704042C6D
:1009400000D904241D1D072D01D2002300E0DB1E69
:10095000012606FA04F56D1E0D409D409E40761E50
:10096000164045EA0601F0BC00F014BE0CED00E0B4
:10097000064A00F0070110684FF6FF03184040EAEE
:100980000120034908431060704700000CED00E0AF
:100990000000FA052DE9F047DFF8BC9104460E4649
:1009A000D9F8000000F00700B0420CD2D9F80010CE
:1009B00021F007013143C9F80010D9F8000000F018
:1009C0000700B0427ED12078DFF89081800707D5FC
:1009D000D8F80010E26821F00F011143C8F80010A8
:1009E0002078C00762D0D8F80010A26821F47061A6
:1009F0001143C8F8001059496068183902281CD002
:100A000003281DD0096801281DD04907002960DA94
:100A1000524F083F396821F0070101433960FFF761
:100A2000F3FE0546606841F28831022813D003289E
:100A30001ED001288A4627D034E009688903E5E7FB
:100A400009688901E2E7C905E0E7FFF7DDFE411B20
:100A5000514501D923E08A463868C0F3C200022814
:100A6000F3D123E0FFF7D0FE411B514501D916E039
:100A70008A463868C0F3C2000328F3D116E0FFF7B6
:100A8000C3FE411B51450AD83868C0F3C200012893
:100A9000F5D10BE0FFF7B8FE411B514502D9032009
:100AA000BDE8F087386810F0380FF3D1D9F800109E
:100AB000484601F00701B1420DD9016821F0070154
:100AC000314300E005E00160006800F00700B0423B
:100AD00001D00120E4E72078400707D5D8F80010BE
:100AE000226921F070011143C8F800102078010735
:100AF0001B4805D50168626921F07001114301604E
:100B00002178C90605D50168A26921F4E061114385
:100B100001602078800607D51149091D0868E2693F
:100B200020F070001043086000F066F8D8F800105C
:100B30004FF4807292FAA2F201F47061B2FA82F27A
:100B4000D140084A515CC840074908600F20FFF7B0
:100B500077FE0020A4E7000000200052184402584D
:100B60001C4402586E1800080000002410B5FFF75E
:100B7000B1FC08490968012292FAA2F201F00F01C2
:100B8000B2FA82F2D140044A515CC840034908607D
:100B900010BD0000184402586E180008040000241C
:100BA00010B5FFF7E3FF07490968102292FAA2F295
:100BB00001F07001B2FA82F2D140034A515CC840A0
:100BC00010BD00001C4402586E18000810B5FFF755
:100BD000CDFF074909684FF4807292FAA2F201F43E
:100BE000E061B2FA82F2D140024A515CC84010BDC5
:100BF0001C4402586E1800083548F0B50068364DA0
:100C000010F03801334809D00411082904D0334EBC
:100C100010290BD018290BD02046F0BD2968890671
:100C2000FBD52968C1F3C101C840F0BD3046F0BD15
:100C3000274918310A68096812F00302284BC1F3EA
:100C400005111B68274F03F001033F68DFED260AFB
:100C5000B7EE001AC7F3CC0717FB03F300EE103A08
:100C6000224BB8EE400A06D0012A01D0022A2BD02E
:100C7000B4FBF1F008E02A68920603D52A68C2F3B3
:100C8000C102D040B0FBF1F001EE900A1868B8EE56
:100C9000612AC0F3080001EE900A1868F8EE611AA4
:100CA00040EE201A31EE810A22EE000AC0F34620FF
:100CB000401C00EE900AF8EE600A80EE201ABCEEAE
:100CC000C10A10EE100AF0BDB6FBF1F0DCE700003F
:100CD000104402580090D0030044025840787D012F
:100CE0002C44025834440258000000393044025861
:100CF0002DE9F05F04460078DFF8FC8341F2883983
:100D0000DFF8F8A3FE4DC0074ED0D8F800104046DB
:100D1000C1F3C20102291AD00068C0F3C20003283F
:100D200005D1DAF8000000F0030002280FD0606857
:100D3000B0F5803F12D010B1B0F5A02F19D02868BF
:100D400020F480302860286820F4802009E028689A
:100D5000800329D56068002874D025E0286840F415
:100D600080302860606890B1FFF74EFD06464F4620
:100D700009E0286840F480202860EFE7FFF744FD91
:100D8000801BB8427DD828688003F7D50CE0FFF7B8
:100D90003BFD06464F4604E0FFF736FD801BB84298
:100DA000F0D828688003F7D42078D64F80075AD52A
:100DB000D8F8001040464FF47C3B11F0380F13D0A8
:100DC0000068C0F3C200032803D1DAF800008007EE
:100DD0000AD0E068A8B3296821F01901014329600D
:100DE000FFF712FD06461DE02868400702D5E068BF
:100DF0000028B1D02868E16820F019000843286075
:100E0000FFF702FD064604E0FFF7FEFC801B022808
:100E1000B8D828684007F7D507E0FFF7F5FC801B36
:100E20000228AFD828684007F7D538689BFAABF29C
:100E300020F47C312069B2FA82F29040014339609B
:100E400011E000E0AEE0286820F001002860FFF724
:100E5000DBFC064604E0FFF7D7FC801B022891D894
:100E600028684007F7D42078C00655D5D8F8001078
:100E700040464FF0F84BC1F3C201012917D000687A
:100E800000E0EDE0C0F3C200032805D1DAF800006D
:100E900000F0030001280AD0E069002828682CD05F
:100EA00040F080002860FFF7AFFC064616E0286897
:100EB000C00502D5E069802874D138689BFAABF28E
:100EC00020F0F841206AB2FA82F290400143396082
:100ED00022E0FFF799FC801B022899D82868C005FA
:100EE000F7D538689BFAABF2216AB2FA82F220F0A9
:100EF000F8409140084338600EE020F08000286000
:100F0000FFF782FC064604E0FFF77EFC801B022808
:100F100087D82868C005F7D42078000724D5774FF4
:100F200060694C37002838680FD040F00100386005
:100F3000FFF76AFC064604E0FFF766FC801B022808
:100F40008DD838688007F7D50EE020F001003860B2
:100F5000FFF75AFC064604E0FFF756FC801B022808
:100F60007ED838688007F7D42078800623D5A0691A
:100F7000002828680FD040F480502860FFF744FC18
:100F8000064604E0FFF740FC801B022868D828686A
:100F90008004F7D50FE020F480502860FFF734FC80
:100FA000064605E0D6E0FFF72FFC801B022857D845
:100FB00028688004F7D42078400744D5524F386819
:100FC00040F480703860FFF71FFC064604E0FFF72E
:100FD0001BFC801B642843D83868C005F7D5474FF1
:100FE000A068483701280AD008B1052811D0386810
:100FF00020F001003860386820F0040002E0386812
:1010000040F001003860A06888B1FFF7FDFB06469C
:1010100009E0386840F004003860F0E7FFF7F4FBBF
:10102000811B49451CD838688007F7D50BE0FFF7CE
:10103000EBFB064604E0FFF7E7FB811B49450FD8B1
:1010400038688007F7D4606AF0B3D8F80010C1F3AD
:10105000C20103297ED00228286820F0807000E0B9
:1010600079E0286003D0FFF7CFFB044687E0FFF765
:10107000CBFB064604E0FFF7C7FB801B02287BD8AA
:1010800028688001F7D4DAF8001040F2F332914377
:10109000E26A41EA0211A26A1143CAF8001094F808
:1010A00034004FF4FE02218E4002491EA0F500706C
:1010B00080B2C1F308010843218F491E02EA0141B1
:1010C000084394F83C1000E05CE0491E120202EA7A
:1010D000016108430949083108600B1D19684FF682
:1010E000F872A06C914392FAA2F2B2FA82F29040A6
:1010F00001431960014809E010440258284402588D
:10110000004402580444025800480258001D016877
:10111000226C21F00C01114301600168626C21F026
:10112000020111430160016841F4803101600168EE
:1011300041F400310160016841F4802101600168DF
:1011400041F001010160286840F080702860FFF7DD
:101150005BFB01E018E00FE0044604E0FFF754FBFE
:10116000001B022808D828688001F7D50AE0FFF79D
:101170004BFB001B022802D90320BDE8F09F286822
:101180008001F4D40020F8E70120F6E74FF0E021D9
:101190000428086903D020F004000861704740F07B
:1011A0000400FAE7401EB0F1807F10B501D30120A2
:1011B00010BD4FF0E02460610F21601700F0EAF9E4
:1011C0000020A06107202061002010BD10B500683C
:1011D00086B01B49884230D11A48016841F00101AC
:1011E0000160006800F001000590164810300168A9
:1011F00041F01001016000680121134C00F0100063
:1012000005904FF4007000900220CDE90101039099
:101210000720694604902046FFF7F4F94FF48061F7
:10122000204600916946FFF7EDF92520FFF773FB93
:10123000032225201146FFF77BFB06B010BD0000FE
:1012400000100140E04402580000025830B5006828
:10125000114988420CD1114A5088010408D4114622
:101260004FF000034404097806D50A2901D05380C1
:1012700030BD40F400400DE00D2909D0084DC0F309
:101280000D04401C80B2C72829555080EFD830BDCE
:1012900040F48040508030BD001001400C0000241C
:1012A0003400002454482DE9F041524C86B00168C6
:1012B00041F002010160016841F0200101604E48E7
:1012C0000C38016841F48041016040200090022008
:1012D00001900320DFF82481002569460A2704973E
:1012E000CDE902504046FFF78DF9042069460926F2
:1012F000049600904046FFF785F90496C020404EC2
:10130000694600903046FFF77DF94FF4407069461A
:10131000049700903046FFF775F937486438016844
:1013200041F480410160016821F48041016031484D
:10133000203881688906FCD4324901603249416015
:10134000016841F00101016081688906FCD44FF415
:101350009C71416181688907FCD5C16841F0020137
:10136000C16081688906FCD44FF483714161816852
:101370008907FCD5C16841F00201C1608168890616
:10138000FCD422494161056181684907FCD53021BF
:101390002170016841F00401016081688907FCD572
:1013A000C16841F00201C16081688906FCD481688E
:1013B0008906FCD4C561164941611648016821F4CB
:1013C00080310160134970310A6822F001020A601D
:1013D0000A1D156082060F4B78331A601B1D0E4ADA
:1013E0001A6005220A60016841F48031016006B08C
:1013F000BDE8F08120500052E04402580004025839
:10140000001402581003000101041600C003000379
:10141000EBEF180F24ED00E02D00030370B5294C0D
:101420009CB0256825F004052560264C00260C3468
:10143000256845F440452560256805F440451B9521
:101440002568AD04FCD5012400940CAD039624045A
:10145000019402240994CDE90A410796082485E8FD
:101460000D00CDE910466846FFF742FC98B9FFF73A
:1014700019FF3F2013900320CDE9140640200101FD
:10148000CDE91640CDE9180150201A90022113A889
:10149000FFF780FA10B101201CB070BD0A48016846
:1014A00041F0800101600848F430016841F0020118
:1014B0000160006800F002001B90FFF79BF800201D
:1014C000EAE700000C480258004402581C48016832
:1014D00041F4700101601B49086840F00100086098
:1014E000184A0020103210600A68174B1A400A6030
:1014F000144A18321060121D1060121D1060114A3B
:1015000028321060121D1060121D1060121D106034
:10151000121D1060121D1060121D1060121D10604F
:101520000A6822F480220A600649603108600120BE
:101530000649C1F80801C0060149803908607047B2
:1015400088ED00E0004402587FEDF6EA008000518B
:1015500070B50D4D00240D48FEF7C1FF02E0641C7C
:10156000AC4204D80948FEF7BFFF2028F7D1002479
:1015700002E0641CAC4206D8054901220348FEF78C
:10158000B8FF0028F5D170BDFFFF0100FC0000246A
:101590000C0000240907090E002804DB00F1E020FC
:1015A00080F80014704700F00F0000F1E02080F890
:1015B000141D70477047000010B504460420FFF763
:1015C000E5FD0148046010BD0800002470B500244A
:1015D00005464FF47A7603E0304600F005F8641CC7
:1015E000AC42F9D370BD000070B54FF0E02500218A
:1015F0006C69094AAB6912685043AA699A42FCD0E7
:1016000002D2A3EB020302E0A4EB02063344194426
:1016100013468142F1D370BD080000240349CA6912
:101620005206FCD5C2B20A85704700000010014086
:101630001CB50024FEF79AFFFFF7F4F804230222FA
:101640000521A020FFF7EAFE4FF4C870FFF7B4FFB2
:101650004FF4E13000F0EAF8FEF750FFFEF753FFD9
:10166000FEF756FFFEF759FF464E4FF4784010251F
:10167000C8222B463221306043A0CDE900501E2005
:10168000FEF750FF45A01023C822CDE900504621A7
:101690001E20FEF747FF44A01023C822CDE90050CA
:1016A0005A211E20FEF73EFF1023C8226E2142A0C1
:1016B0000FE044A01023C822CDE9005082211E2053
:1016C000FEF730FFC820FFF781FF1023C8228221D8
:1016D00040A0CDE900501E20FEF724FFFEF727FFB3
:1016E0000028E6D13FA01023C822CDE90050822176
:1016F0001E20FEF717FF3FA01023C822CDE900509F
:1017000096211E20FEF70EFF3FA01023C822CDE930
:101710000050B4211E20FEF705FF3EA01023C82272
:10172000CDE90050D2211E20FEF7FCFE3E4F1F20C7
:10173000306014260020FEF7FFFE012808D1FEF7D6
:1017400000FF0A230246B42100957620FEF7FEFE34
:10175000B4FBF6F006FB104070B902213846FFF7E3
:101760004AF809210020FEF7F6FE01230246D221A5
:1017700000959E20FEF7EAFE0A20FFF727FF641C73
:10178000E4B2D7E724000024504F4C415249532083
:10179000483735302F46373530000000524E47204D
:1017A000544553540000000041544F4D40414C49B2
:1017B000454E54454B000000323031392F342F3222
:1017C000380000002020524E47204572726F72216F
:1017D00020000000524E4720547279696E672E2E09
:1017E0002E000000524E472052656164792120206E
:1017F000200000004B4559303A4765742052616E15
:10180000646F6D204E756D0052616E646F6D204E79
:10181000756D3A0052616E646F6D204E756D5B3070
:101820002D395D3A00000000000402580B490A4AB5
:1018300010B5C1E9002000208860C8600861886197
:101840000C2048610846FEF78BFEBDE810400449B5
:1018500001220248FEF74DBE00100140FC000024AA
:101860000C0000244FF04070E1EE100A70470000B9
:101870000000010203040102030406070809000036
:10188000A01800080000002434000000D402000862
:10189000D418000834000024140F0000F0020008DF
:1018A0000090D0030090D003000000000000000072
:1018B0000000000001000000100000000000000017
:1018C00001000000000000FFFFFFFFFF000000001C
:0418D0000000000014
:0200000490006A
:10000000782900F043800020704700000FB40449B5
:1000100010B503AA029800F0F1F810BC5DF814FBCB
:10002000100000242DE9F0410E4604460020206215
:100030002046E168884730B3252805D0D4E901215E
:100040009047206A401CF2E7E16820460027884775
:10005000050018D0A5F14100192802D820354FF429
:1000600000673246294620462760FFF7C9FF40B1A6
:10007000012804D0F61D26F007060836D8E7361DFD
:10008000D6E72846DAE7206ABDE8F08170B5044675
:100090000D4621461068AFF300802188090502D57E
:1000A0000F4A7A4402E00E4A7A440E32002104F1EB
:1000B000240305E000F00F060009965D5E54491C1C
:1000C0000028F7D120780023000704D5702D02D036
:1000D00009B1022311322046BDE8704000F034B867
:1000E000FE9E000010B5203AC0F00B80B1E8185019
:1000F000203AA0E81850B1E81850A0E81850BFF412
:10010000F5AF5FEA027C24BFB1E81850A0E81850B0
:1001100044BF18C918C0BDE810405FEA827C24BF04
:1001200051F8043B40F8043B08BF7047D20728BF92
:1001300031F8023B48BF11F8012B28BF20F8023BE1
:1001400048BF00F8012B70472DE9F0470D4699464E
:100150009246044600F124080168880604D5E06947
:1001600021F01001216000E00120A84201DD471BC1
:1001700000E00027A1697A1902EB0900081AA061C2
:100180002078C00602D42046AFF30080002608E0A5
:10019000D4E901211AF806009047206A401C761C19
:1001A00020624E45F4DB2078C0060AD52046AFF326
:1001B000008006E0D4E9012130209047206A401CED
:1001C0002062381EA7F10107F4DC07E0D4E9012121
:1001D00018F805009047206A401C2062281EA5F1EF
:1001E0000105F3DC2046AFF300802078000602D53D
:1001F0000220BDE8F0870120FBE70000074B70B547
:100200000D467B4400F011F80446284600F020F823
:1002100010B14FF0FF3070BD204670BD171400784C
:1002200001694A1C02610878704700B58FB0CDE9BA
:1002300001310021059105497944CDE903101146AA
:100240006846FFF7EFFE0FB000BD0000E5FFFFFFBF
:10025000007B00F08000704740F2056CC0F6000C97
:10026000604740F6F93CC0F6000C604740F66D3C34
:10027000C0F6000C604740F6090CC0F6000C604761
:1002800041F2CD1CC0F6000C604740F2ED7CC0F698
:10029000000C604741F2CD5CC0F6000C604741F2B3
:1002A000E95CC0F6000C604740F2FF7CC0F6000C31
:1002B000604740F6D50CC0F6000C604740F6810C54
:1002C000C0F6000C604740F6F10CC0F6000C604729
:1002D00040F6150CC0F6000C604741F24D2CC0F6FC
:1002E000000C604740F27B3CC0F6000C604740F6D3
:1002F000A13CC0F6000C604740F6CD3CC0F6000CB7
:100300006047FEE77047000070B5B3F5804F05D039
:100310006FF0704140F82210002070BD50F822307C
:10032000084C2340D1E900458E8944EA05148D68C4
:1003300089692D0245EA06452C430C431C4340F8CD
:100340002240E9E70000F0CFF0B50C6850F82450E7
:100350001A4A1540D1E90123D1E903671A433E4304
:1003600032434E6932438E693243CE6932430E6A5C
:1003700032434E6A32438E6A3243CE6A32430E6B48
:1003800032438E6B32434E6B32432A43082B01D1EA
:1003900042F0400240F824200A6BB2F5801F05D1DC
:1003A0000A684AB1026842F4801202600A681AB10F
:1003B0000268496B0A4302600020F0BD8004C0FF60
:1003C00000EB8202F0B553688E8903F04044D1E916
:1003D000003543EA05138D682D0245EA06450E8A6D
:1003E0002B430D4D05EB065633430E7D6F0107EB96
:1003F000066633438E693343234353600268D20257
:1004000007D54268098A22F4700205EB01511143B5
:1004100041600020F0BD00000000F0FF30B5D1E9E0
:1004200001230D681A43D1E9033423431A434B696E
:100430001A438B691A43D1E90734496A012D0568CB
:1004400007D01A4322430A436FF30E052A43026082
:100450000AE025F4F845234329430B434168036030
:100460006FF30E010A434260002030BD426942EA48
:10047000410141610020704718B5D1E900236FF0B8
:100480001F041A438B68C96804EB431343EA4121F4
:100490000A4300920261002018BD0000F0B5D1E9C6
:1004A00000346FF00F055B1E2E0105EB041423438F
:1004B0008C682F034FEA054C0D8A06EB04248E8AC4
:1004C0002343CC68097E4FF07F4E012A07EB054598
:1004D0000CEB06560EEB01610CD082683F1107EB66
:1004E000043423432B4333430B4302F07042134342
:1004F00083600FE08768084A17402203C468A2F5AA
:10050000805232433A4382602B430B4304F07044E1
:100510002343C3600020F0BDFF0F0FFF10B528B1CB
:1005200090F83510022903D080214165012010BDCB
:100530001D4A4FF4956301688C189C4207D8042229
:1005400080F83520086820F00100086029E00C6878
:1005500024F00E040C6001680A440A6822F00102CB
:100560000A60016E0A6822F480720A6090F85C30BA
:10057000012202FA03F10D4B1960D0E919134B6007
:10058000C16E31B10B6823F480730B60D0E91C138A
:100590004B60002180F8341080F83520016D01B1E6
:1005A0008847002010BD0000F0FFFDBF0454025832
:1005B0002DE9F041044690F8A00015460F460128A9
:1005C0001DD0012684F8A060022084F8A10005EB6C
:1005D000850000EBC500342204EB80003830FFF7C3
:1005E00081FD2A463946204604F034FB20684662E5
:1005F00084F8A160002084F8A000BDE8F08102200A
:10060000FBE7000070B5040004D094F8A1000025B9
:1006100010B106E0012070BD204684F8A05000F023
:100620006BF8022084F8A1002068816921F07041F4
:100630008161D4E901100143D4E90302104301436D
:1006400020688269114381612068826829490A40D3
:100650008260A08A020420688368A669334313433A
:1006600083602068C2680A40C260A08B02042068D0
:10067000C368266A33431343C360206802690A4093
:100680000261A08C020420680369A66A3343134305
:100690000361206842690A404261A08D010420681C
:1006A0004269236B1A430A43426194F835000202FF
:1006B00094F8360001042068C36A03F07F43C362E4
:1006C0002068C36A114394F8346033430B43C36218
:1006D0002068416B41F0060141632068816941F067
:1006E00001018161C4F8A450012084F8A100002018
:1006F00070BD000000F800F02B4810B586B001680E
:1007000041F008010160006800F0080005902648EB
:100710001038016841F010010160006800F010001D
:1007200005902148001F016841F480710160016853
:1007300001F480710591016841F400710160016864
:1007400001F400710591016841F480610160006865
:100750000324694600F48060059020200090012069
:100760000190CDE902041148FFF776FD4FF4E04017
:1007700000900220019000206946CDE902040E207D
:1007800004900B48FFF768FD48F67C60009009482C
:100790006946FFF761FDFF20009007486946FFF7B3
:1007A0005BFD06B010BD0000E4440258000402588E
:1007B00000200258002402580028025870B5044650
:1007C00090F8A0000E46012820D0012584F8A05002
:1007D000022084F8A10003EB830000EBC30004EBCC
:1007E00080018E63086E3044C1E90F02486E1044E8
:1007F000486438311A46204604F02CFA20684562D5
:1008000084F8A150002084F8A00070BD022070BDC3
:1008100070B5044690F8A0000E46012820D00125AE
:1008200084F8A050022084F8A10003EB830000EBC1
:10083000C30004EB8001886B3044C863086C10442B
:100840004864C1E9186238311A46204604F002FAB9
:100850002068456284F8A150002084F8A00070BD93
:10086000022070BD10B5FFF7FCFC084909684FF481
:10087000807292FAA2F201F47061B2FA82F2D1406F
:10088000034A515CC8400349086010BD184402582F
:100890006E1800080000002410B5FFF7E7FC0749B8
:1008A0000968102292FAA2F201F07001B2FA82F203
:1008B000D140034A515CC84010BD0000204402589A
:1008C0006E180008364930B50A68096812F003024C
:1008D000344BC1F305311B68334C03F0100324681B
:1008E000DFED320AB7EE001AC4F3CC0414FB03F3B5
:1008F00000EE103A2E4BB8EE400A07D02D4C012ADC
:1009000001D0022A4AD0B4FBF1F10BE0244C283C80
:1009100022689506284A03D52468C4F3C104E2403E
:10092000B2FBF1F101EE901A1968B8EE612AC1F339
:10093000080101EE901A1968F8EE611A40EE201ACB
:1009400031EE810A22EE000AC1F34621491C00EE75
:10095000901AF8EE600A80EE201AFCEEC10AC0ED93
:10096000000A1968C1F30641491C00EE901AF8EE1E
:10097000600A80EE201AFCEEC10AC0ED010A196877
:10098000C1F30661491C00EE901AF8EE600A80EE91
:10099000201ABCEEC10A80ED020A30BD074ABFE74B
:1009A000284402582C4402583C44025800000039A4
:1009B0003844025800093D000090D00340787D0182
:1009C000364930B50A68096812F00302344BC1F3A6
:1009D00005511B68334C03F480732468DFED320A41
:1009E000B7EE001AC4F3CC0414FB03F300EE103A84
:1009F0002E4BB8EE400A07D02D4C012A01D0022A16
:100A00004AD0B4FBF1F10BE0244C283C2268950657
:100A1000284A03D52468C4F3C104E240B2FBF1F1D3
:100A200001EE901A1968B8EE612AC1F3080101EECF
:100A3000901A1968F8EE611A40EE201A31EE810A18
:100A400022EE000AC1F34621491C00EE901AF8EE8E
:100A5000600A80EE201AFCEEC10AC0ED000A196897
:100A6000C1F30641491C00EE901AF8EE600A80EED0
:100A7000201AFCEEC10AC0ED010A1968C1F3066133
:100A8000491C00EE901AF8EE600A80EE201ABCEEC7
:100A9000C10A80ED020A30BD074ABFE72844025868
:100AA0002C44025844440258000000394044025883
:100AB00000093D000090D00340787D012DE9F84FFA
:100AC0000446006800252E46010104F12400FE4F73
:100AD000DFF8F88300901DD5606E50B1B0F5801F2F
:100AE0000CD0B0F5001F0ED0B0F5401F1DD0012571
:100AF0000FE0386840F40030386016E00221201D15
:100B000004F05CF903E00098022104F0CFF905003D
:100B10000BD02E462088C00523D5606D05281ED237
:100B2000DFE800F00C11161B1B00D8F80010626EF5
:100B300021F440111143C8F80010EBE7386840F485
:100B40000030386009E00021201D04F037F903E08F
:100B50000098002104F0AAF905466DB100E00125D6
:100B60002E432088800528D5A06D80281ED00CDC5F
:100B700090B140280ED114E0D8F80010626D21F039
:100B800007011143C8F80010EBE7C02813D0B0F5F7
:100B9000807F10D001250FE0386840F400303860C5
:100BA00009E00021201D04F009F903E0009800216C
:100BB00004F07CF9054685B12E432088DFF81093B8
:100BC00040052CD5D4F8A400B0F5800F20D00DDC62
:100BD000A0B1B0F5001F0FD115E0D8F80010A26D3C
:100BE00021F4E0711143C8F80010E6E7B0F5C00F3A
:100BF00013D0B0F5000F10D001250FE0386840F495
:100C00000030386009E00021201D04F0D7F803E02F
:100C10000098002104F04AF9054675B12E4320885A
:100C200000052DD5D4F8A800B0F1007F21D00EDC4E
:100C3000A8B1B0F1807F10D116E0D9F80010D4F837
:100C4000A42021F460011143C9F80010E7E7B0F1D6
:100C5000407F13D0B0F1806F10D001250FE03868CD
:100C600040F40030386009E00021201D04F0A6F8AF
:100C700003E00098002104F019F905466DB12E43F8
:100C8000206880011FD5A06CD8B110280FD0202873
:100C900012D0302815D0012514E0D9F80010D4F86E
:100CA000A82021F0E0611143C9F80010E8E7386896
:100CB00040F40030386004E00221201D04F07EF88A
:100CC00005466DB12E432088C0042BD5E06DB0F5EC
:100CD000005F20D00DDCA0B1B0F5805F0FD115E032
:100CE0007A48001F0168A26C21F0300111430160B5
:100CF000E9E7B0F5405F13D0B0F5804F10D0012583
:100D00000FE0386840F40030386009E00021201D11
:100D100004F054F803E00098002104F0C7F80546F9
:100D200085B12E432088800429D5206EB0F5403F40
:100D300023D010DC08B3B0F5803F14D0B0F5003FED
:100D40000FD115E0D8F80010E26D21F4E041114315
:100D5000C8F80010E6E7B0F5802F0ED0B0F5A02F50
:100D60000BD001250AE00121201D04F027F803E043
:100D70000098012104F09AF805468DB12E43208891
:100D800040042AD5D4F8AC00B0F1405F23D010DC89
:100D900008B3B0F1805F14D0B0F1005F0FD115E05F
:100DA000D8F80010226E21F4E0211143C8F8001099
:100DB000E5E7B0F1804F0ED0B0F1A04F0BD0012588
:100DC0000AE00121201D03F0F9FF03E00098012152
:100DD00004F06CF805466DB12E43208800041FD541
:100DE000E06ED8B1B0F1805F0ED0B0F1005F10D0EE
:100DF000012514E0D9F80010D4F8AC2021F0E0412E
:100E00001143C9F80010E8E7386840F40030386052
:100E100004E00121201D03F0D1FF05466DB12E43F2
:100E20002068C0011ED5606CD0B101280ED0022808
:100E300011D0032814D0012513E0D8F80010E26E79
:100E400021F040511143C8F80010E9E7386840F438
:100E50000030386004E00221201D03F0AFFF05469A
:100E600075B12E432068DFF86CB040025AD51A489D
:100E7000016841F480710160FFF7FDF982460EE0E0
:100E80001248001F0168626C21F0030111430160E8
:100E9000E8E7FFF7F0F9A0EB0A0064283AD80E481B
:100EA0000068C005F5D5B5BB094818300068B4F82E
:100EB000B01000F4407001F44071884219D0044829
:100EC000183001680AE000002C44025850440258CF
:100ED000584402581044025800480258026821F44D
:100EE000407142F480320260026822F48032026073
:100EF0000160D4F8B000B0F5807F22D1FFF7BBF9D4
:100F0000824609E0FFF7B7F9A0EB0A0141F2883009
:100F1000814201D9032504E0FE4800688007F1D52D
:100F20007DB12E432078DFF8F0A3C0073CD0A06F3E
:100F3000182837D025DC78B3082828D0102824D1E9
:100F40002BE0D4F8B000C0F3012103290ED0DBF868
:100F5000001021F47C51CBF80010EE480168B4F881
:100F6000B020C2F30B0211430160DBE7DBF8002085
:100F7000EA4B22F47C5203EA10100243CBF8002023
:100F8000EBE720280ED028280CD001250BE001210A
:100F9000201D03F013FF04E004E00098012103F09A
:100FA00085FF05465DB12E43207880071ED5606F12
:100FB000062819D2DFE800F0160C11161616DAF81A
:100FC0000010A26F21F038011143CAF80010EBE7BE
:100FD0000121201D03F0F2FE03E00098012103F03F
:100FE00065FF054675B100E001252E4320784007D6
:100FF0001FD5D4F89000062819D2DFE800F0160CAF
:1010000011161616DAF80010626F21F0070111436D
:10101000CAF80010EAE70121201D03F0CFFE03E02B
:101020000098012103F042FF05469DB100E0012533
:101030002E43207880062BD5D4F88C00B0F1405F89
:1010400024D011DC10B3B0F1805F15D0B0F1005F97
:1010500010D116E0D9F80010D4F8902021F0070143
:101060001143C9F80010E4E7B0F1804F0ED0B0F1A1
:10107000A04F0BD001250AE00021201D03F09EFEA9
:1010800003E00098022103F011FF05468DB12E43C5
:10109000207840062BD5D4F89800B0F5406F24D0C6
:1010A00011DC10B3B0F5806F15D0B0F5006F10D122
:1010B00016E0DAF80010D4F88C2021F0E04111435A
:1010C000CAF80010E4E7B0F5805F0ED0B0F5A05F7D
:1010D0000BD001250AE00021201D03F06FFE03E084
:1010E0000098022103F0E2FE05468DB12E432078E0
:1010F00000062BD5D4F89C00B0F5C04F24D011DCED
:1011000010B3B0F5005F15D0B0F5804F10D116E0E8
:10111000D9F80010D4F8982021F4E0511143C9F80F
:101120000010E4E7B0F5004F0ED0B0F5204F0BD023
:1011300001250AE00021201D03F040FE03E0009895
:10114000022103F0B3FE054665B32E432078000765
:101150000BD5D4F88000B0F5805F2DD0DAF80020F0
:1011600022F440520243CAF800202078C0060BD572
:10117000D4F89400B0F5807F24D0D9F8002022F470
:1011800040720243C9F80020206800032CD5D4F82F
:10119000A000E8B1B0F5803F1FD0B0F5003F21D0EE
:1011A000012520E0D9F80010D4F89C2021F46041FA
:1011B0001143C9F80010C9E70098022103F076FE38
:1011C0000643D2E70098022103F070FE0643DBE7F6
:1011D0000021201D03F0F2FD03E00098022103F03E
:1011E00065FE054685B12E432068400322D5D4F81C
:1011F0008400B0F5801F11D0B0F5001F13D0B0F5FA
:10120000401F15D0012514E0D9F80010D4F8A02013
:1012100021F440311143C9F80010E5E7386840F483
:101220000030386004E00098012103F03FFE0546DD
:1012300055B12E432068C0031CD5E06C70B1B0F5E9
:10124000803F10D0012514E0DAF80010D4F8842093
:1012500021F440111143CAF80010EBE7386840F45C
:101260000030386004E00221201D03F0A7FD054690
:10127000C5B12E432068800004D50098022103F0F8
:1012800015FE0643206880031BD5E06FB8B1B0F5AA
:10129000807F10D0B0F5007F11D0B0F5407F0ED028
:1012A00001250DE01C4808380168E26C21F480310A
:1012B00011430160DEE7386840F40030386045B320
:1012C0002E432068C00207D5D8F80000226F20F016
:1012D00000401043C8F800002068C00008D5DBF8C3
:1012E0000010D4F8B42021F480411143CBF8001051
:1012F0002068800207D5D8F80010A26E21F0807116
:101300001143C8F800102068400014D5DBF8001025
:1013100006E01EE07044025854440258CFFFFF001C
:1013200021F40041CBF80010DBF80010D4F8B8200D
:101330001143CBF800102068002806DA0A4801683B
:10134000226D21F04051114301605EB10120BDE8E2
:10135000F88FDAF80010E26F21F440711143CAF8F7
:101360000010AEE70020F2E74C44025810B504002C
:1013700010D02068016821F02C01016020684168CC
:1013800021F060014160204600F058F800206072B2
:10139000207210BD012010BD2DE9F0470446007AEF
:1013A0000026894601280BD001272772607AB046B3
:1013B000012807D0012684F808803046BDE8F08770
:1013C0000220FBE702206072FEF755FF05460AE0A7
:1013D000FEF751FF401B022805D90420607203204C
:1013E00084F80880EAE720684068C043C007EFD16E
:1013F00020688068E060C9F800006772DBE710B51C
:10140000040002D0607A10B106E0012010BD002077
:101410002072204600F014F80220607220680168F3
:10142000626821F02001114301602068016841F0E9
:101430000401016001206072002010BD70470000AF
:1014400000B5B1B04FF40030009040121F906846D4
:10145000FFF734FB0548016841F040010160006876
:1014600000F040002F9031B000BD0000DC44025875
:1014700070B504000D4603D094F82C0010B107E0BD
:10148000012070BD002084F82D00204600F018F8DF
:10149000022084F82C002068211DFEF7BFFFD4E94C
:1014A00000022946FEF7FAFF0448016841F00041B6
:1014B0000160012084F82C00002070BD0040005223
:1014C000444800B587B0016841F00201016000683E
:1014D00000F0020005903F482038016841F4805137
:1014E0000160006800F4805005903A4814380168A3
:1014F00041F004010160016801F0040105910168F7
:1015000041F008010160016801F0080105910168DE
:1015100041F010010160016801F0100105910168BE
:1015200041F020010160016801F02001059101688E
:1015300041F040010160016801F04001059101683E
:1015400041F080010160016801F0800105910168AE
:1015500041F4807101600068694600F48070059074
:101560000D200090022001900120029003200390A2
:101570000C2004901848FEF76FFE4CF203700090A8
:1015800016486946FEF768FE4FF6837000901448CF
:101590006946FEF761FE4FF63F000090114869462C
:1015A000FEF75AFE48F2371000900F486946FEF7E2
:1015B00053FE4FF47F4000900C486946FEF74CFE06
:1015C00040F2FF6000900A486946FEF745FE07B00A
:1015D00000BD0000F444025800080258000C0258F4
:1015E000001002580014025800180258001C02583B
:1015F0000020025810B5044690F82C00022809D0AB
:10160000022084F82C002068FEF730FF012084F8C7
:101610002C00002010BD70B5044690F82C000D463B
:1016200002280CD0022084F82C002068FEF724FF4A
:101630002868022804D0012084F82C00002070BD06
:101640000520F9E770B5040015460E4603D094F85E
:10165000450010B107E0012070BD002084F844006F
:10166000204600F021F8206804F10801FEF76CFE26
:10167000A26831462068FEF7A3FEE36A2946D4E952
:101680000102FEF741FEA168206850F8212042F0D7
:10169000010240F821200348016841F00041016047
:1016A000002070BD004000521A4800B587B00168A4
:1016B00041F480510160006800F4805005901548A5
:1016C0000C30016841F008010160016801F0080177
:1016D0000591016841F0100101600068694600F061
:1016E000100005904EF2B37000900220019001208E
:1016F0000290032003900C2004900748FEF7ACFDF5
:101700004FF68070009005486946FEF7A5FD07B0CA
:1017100000BD0000D4440258000C025800100258CA
:101720007047704790F8791090F87A000843704736
:1017300070B502680446D0691368916810F00F0F05
:1017400064D0594D03F490760D40354376D0C507EB
:1017500007D0DD0505D501251562E26F42F00102D3
:10176000E267820708D5CA0706D0256802222A62E6
:10177000E26F42F00402E267420708D5CA0706D0CA
:10178000256804222A62E26F42F00202E267020741
:101790000ED503F0200201F080552A4352EAC172AF
:1017A00006D0256808222A62E26F42F00802E2674A
:1017B000E26F002A3AD0800608D503F0200001F03D
:1017C0008051084302D0204603F045FDE06F00073A
:1017D00003D42068806840062AD5204603F02DFDFA
:1017E0002068816849061ED5816821F0400181602A
:1017F000606FC0B12D490165606FFEF78FFE002854
:1018000014D0606F016DBDE870400847850615D59E
:1018100003F0200501F0805635430FD02046BDE887
:10182000704003F018BD2046FFF77BFF70BD05E058
:101830002046FFF776FF0020E067F7E7C6024FF08B
:1018400020050CD54E020AD5E803106284F87950C1
:1018500084F87A502046BDE87040FFF761BF060665
:101860000AD503F0800601F400010E4304D020469F
:10187000BDE8704003F07EBF41060BD5590609D57F
:101880001168204621F04001116084F8795000F081
:1018900097F8CBE70002C9D55800C7D5106820F0EB
:1018A00080401060C2E70000010000102752009045
:1018B00010B5040003D094F8790010B107E00120BE
:1018C00010BD002084F878002046FEF7D9FC2420C3
:1018D00084F879002068016821F001010160204648
:1018E00003F0F4FC0128EBD0606B10B1204603F04C
:1018F00008FC2068416821F49041416020688168BB
:1019000021F02A0181602068016841F00101016035
:101910002046BDE8104003F058BC90F87A30202BE8
:101920004CD1B9B1B2B190F87830012B46D0012337
:1019300080F878304166A0F86820A0F86A20FF227D
:101940008168B1F5805F07D07F2351B1B1F1805F2D
:101950000CD010E001207047016921B940F2FF115D
:1019600007E0016909BBA0F86C2004E00169E1B15E
:101970003F21A0F86C100021C167222280F87A2054
:1019800080F8781001688A6842F001028A60016874
:101990000A6892000CD50A6842F480720A600068F6
:1019A000816841F08051816006E0A0F86C30E2E788
:1019B000086840F49070086000207047022070476B
:1019C0007047FEE71B4870B586B0016841F0010121
:1019D0000160016801F001010591016841F0040115
:1019E0000160016801F004010591016841F0800186
:1019F0000160006803240025694600F0800005901E
:101A000002200126CDE902040B48CDE90065FEF76E
:101A100023FC700303948DE8610008486946FEF7D3
:101A20001BFC0C20009006486946FEF715FC06B02A
:101A300070BD0000E044025800000258000802583F
:101A4000001C02582DE9F0470126304CDFF8C08019
:101A5000DFF8C0907703304D01281DD02078A0B169
:101A600008212846FEF711FCC0B104212846FEF7E4
:101A70000CFC98B139464046FEF707FC70B10121D5
:101A80004846FEF702FC012808D008212846FEF748
:101A9000FCFB012826D037E02670E1E70A20FEF79C
:101AA000F9FB0020207008212846FEF7EEFB80B1EC
:101AB00004212846FEF7E9FB70B139464046FEF79F
:101AC000E4FB58B101214846FEF7DFFB012807D0AF
:101AD0001AE00120BDE8F0870220FBE70320F9E7C8
:101AE0000420F7E704212846FEF7CFFB01280BD19D
:101AF00039464046FEF7C9FB012805D10121484679
:101B0000FEF7C3FB00B926700020E3E720000024A5
:101B10000008025800000258001C02580E490F4AE3
:101B200070B5064608881268002422B13046BDE828
:101B3000704002F0C3BD4D8800214543084602F0C5
:101B400017FC02F083FDB1B2054801E00180641C7E
:101B5000AC42FBD370BD0000C8010024B4020024D5
:101B6000000008602DE9F05F394C3A4DA0712968FA
:101B700039B102F0C7FDE88A2080288B6080BDE87B
:101B8000F09F33492C232A254FF0F0092B2649F2E8
:101B9000413A4FF4305E45F2105B89884FF4487744
:101BA0004FF4A07845F2103C4FF4F07258B1A4F80D
:101BB00000805145A4F8029001D0614529D12381CC
:101BC0006581A68139E0A4F800905145A4F802800F
:101BD00001D0614508D1238161456581A68131D15C
:101BE000A4F8008062802DE0594508D1A4F808E0EF
:101BF0004FF4285060814FF42C50A08106E0A1F5ED
:101C0000C85063381ED123816681A58122806780F8
:101C100018E0594508D1A4F808E04FF42850608135
:101C20004FF42C50A08106E0A1F5C850633804D1D0
:101C300023816581A68127806280614502D122804F
:101C4000A4F802800020BDE8F05F02F0B5BA000001
:101C5000C8010024B40200242DE9F04104463A48AA
:101C60000D46006820B12046BDE8F04102F05EBD9F
:101C7000364E270A4FEA15283146B0884989A0F523
:101C80001343413B0CD0A0F5A643103B08D0A0F570
:101C9000AA43103B11D0A0F5C853633B27D04BE0BB
:101CA000084602F0C7FC384602F0B8FCE0B202F089
:101CB000B5FCB08902F0BEFC38E0084602F0BAFC80
:101CC000384602F0ABFC7089401C80B202F0B2FCD6
:101CD000E0B202F0A3FCB08902F0ACFC404602F096
:101CE0009DFCB089401C80B202F0A4FC21E0B079D8
:101CF00018B93088001B401E84B2084602F09AFCD6
:101D0000270A384602F08AFCE0B202F087FC384627
:101D100002F084FCE0B202F081FCB08902F08AFC9F
:101D2000404602F07BFCE8B202F078FC404602F04C
:101D300075FCE8B202F072FC054930890880881C05
:101D40000280BDE8F0810000B4020024C801002434
:101D5000FEFF07602DE9F04F95B002F01DFFFE4D2C
:101D60004FF6FF7A49F2413945F21036A5F14C0899
:101D700045F2105441F66317A88018B102F04AFDED
:101D800002F08DB9F548016841F002010160006878
:101D90000EA900F00200139020200E9001200F9059
:101DA000109003201190EE48FEF756FA02F0A4F9C5
:101DB000EC491022C8F800104046EB49C8F804105E
:101DC0000021C8F80810C8F80C10C0E9041212026B
:101DD000C8F81810C8F81C10C0E908129200C0E931
:101DE0000A129201C8F830101120C8E90D12CDE98D
:101DF00007015520099015200290CDE90001D64831
:101E00006A460D914C38069107A9FFF71BFC32205A
:101E1000FEF740FAD32002F00DFC02F099F9A880F9
:101E200002F096F9A88002F093F90AEA00205246DF
:101E3000A88002F08DF9A9880843A880484546D0BB
:101E4000D42002F0F7FB02F083F9A88002F080F9B9
:101E5000A88002F07DF902EA0020A88002F078F95B
:101E6000A9880843A880B04231D04FF45A4002F00C
:101E7000E1FB02F06DF9A8804FF45B4002F0DAFB61
:101E800002F066F902EA0020A8804FF45C4002F0FC
:101E9000D1FB02F05DF9A9880843A880B0F5004F96
:101EA0007DD0A04213D0A12002F0C4FB02F050F973
:101EB000A88002F04DF902EA0020A88002F048F95B
:101EC000A9880843A880A0F5AE41613968D080B2E6
:101ED000484566D1CF2002F0ADFB002002F09EFB0A
:101EE000C12002F09BFB302002F098FBED2002F0B5
:101EF000A1FB642002F092FB032002F08FFB122072
:101F000002F08CFB812002F089FBE82002F092FBBA
:101F1000852002F083FB102002F080FB7A2002F083
:101F20007DFBCB2002F086FB392002F077FB2C20D2
:101F300002F074FB002002F071FB342002F06EFB13
:101F4000022002F06BFBF72002F074FB202002F06D
:101F500065FBEA2002F06EFB002002F05FFB002030
:101F600002F05CFBC02002F065FB1B2002F056FB78
:101F7000C12002F05FFB012002F050FBC52002F0FF
:101F800059FB302002F04AFB302002F047FBC7200B
:101F900002F050FBB72002F041FB362002E0B4E033
:101FA000B0E0B4E002F046FB482002F037FB3A20F4
:101FB00002F040FB552002F031FBB12002F03AFB69
:101FC000002002F02BFB1A2002F028FBB62002F0C2
:101FD00031FB0A2002F022FBA22002F01FFBF220BC
:101FE00002F028FB002002F019FB262002F022FB61
:101FF000012002F013FBE02002F01CFB0F2002F096
:102000000DFB2A2002F00AFB282002F007FB082023
:1020100002F004FB0E2002F001FB082002F0FEFAA1
:10202000542002F0FBFAA92002F0F8FA432002F053
:10203000F5FA0A2002F0F2FA0F2002F0EFFA00207F
:1020400002F0ECFA002002F0E9FA002002F0E6FAD1
:10205000002002F0E3FAE12002F0ECFA002002F0A6
:10206000DDFA152002F0DAFA172002F0D7FA07207D
:1020700002F0D4FA112002F0D1FA062002F0CEFAD2
:102080002B2002F0CBFA562002F0C8FA3C2002F0D6
:10209000C5FA052002F0C2FA102002F0BFFA0F20A4
:1020A00002F0BCFA3F2002F0B9FA3F2002F0B6FA83
:1020B0000F2002F0B3FA2B2002F0BCFA002002F04D
:1020C000ADFA002002F0AAFA012002F0A7FA3F20A0
:1020D00002F0A4FA2A2002F0ADFA002002F09EFAE3
:1020E000002002F09BFA002002F098FAEF2002F0A4
:1020F00095FA112002F09EFA7820FEF7CBF82920FD
:1021000001F010BFAF8001F012BFAC80FDE3B04220
:102110007ED1ED2002F08EFA012002F07FFAFE203F
:1021200002F07CFAEE2002F085FADE2002F076FA68
:10213000212002F073FAF12002F07CFA012002F073
:102140006DFADF2002F076FA102002F067FAC42060
:1021500002F070FA8F2009E0C8010024E044025820
:1021600000040258004000520441005202F056FAA6
:10217000C62002F05FFA002002F050FAE22002F0DE
:102180004DFAE22002F04AFAE22002F047FABF20BC
:1021900002F050FAAA2002F041FAB02002F04AFA06
:1021A0000D2002F03BFA002002F038FA0D2002F078
:1021B00035FA002002F032FA112002F02FFA002046
:1021C00002F02CFA192002F029FA002002F026FA77
:1021D000212002F023FA002002F020FA2D2002F044
:1021E0001DFA002002F01AFA3D2002F017FA002032
:1021F00002F014FA5D2002F011FA002002F00EFA4B
:102200005D2002F00BFA002002F008FAB12000E095
:10221000FEE302F00FFA802002F000FA002002F044
:10222000FDF98B2002F0FAF9002002F0F7F9962070
:1022300002F0F4F9002002F0F1F9B22002F0FAF90C
:10224000002002F0EBF9002002F0E8F9022002F091
:10225000E5F9002002F0E2F9032002F0DFF90020A6
:1022600002F0DCF9B32002F0E5F9002002F0D6F923
:10227000002002F0D3F9002002F0D0F9002002F093
:10228000CDF9002002F0CAF9002002F0C7F90020C1
:1022900002F0C4F9002002F0C1F9002002F0BEF9FA
:1022A000002002F0BBF9002002F0B8F9002002F093
:1022B000B5F9002002F0B2F9002002F0AFF90020D9
:1022C00002F0ACF9002002F0A9F9002002F0A6F912
:1022D000002002F0A3F9002002F0A0F9002002F093
:1022E0009DF9002002F09AF9002002F097F90020F1
:1022F00002F094F9002002F091F9B42002F09AF96A
:102300008B2002F08BF9002002F088F9962002F071
:1023100085F9002002F082F9A12002F07FF9002067
:1023200002F07CF9B52002F085F9022002F076F97E
:10233000002002F073F9032002F070F9002002F08F
:102340006DF9042002F06AF9002002F067F9B62066
:1023500002F070F9002002F061F9002002F05EF94D
:10236000B72002F067F9002002F058F9002002F0CF
:1023700055F93F2002F052F9002002F04FF95E209B
:1023800002F04CF9002002F049F9642002F046F90D
:10239000002002F043F98C2002F040F9002002F006
:1023A0003DF9AC2002F03AF9002002F037F9DC20C8
:1023B00002F034F9002002F031F9702002F02EF919
:1023C000002002F02BF9902002F028F9002002F002
:1023D00025F9EB2002F022F9002002F01FF9DC20A1
:1023E00002F01CF9002002F019F9B82002F022F9DD
:1023F000002002F013F9002002F010F9002002F092
:102400000DF9002002F00AF9002002F007F900207F
:1024100002F004F9002002F001F9002002F0FEF8B9
:10242000BA2002F007F9242002F0F8F8002002F0A8
:10243000F5F8002002F0F2F8002002F0EFF8C120D9
:1024400002F0F8F8202002F0E9F8002002F0E6F8A7
:10245000542002F0E3F8002002F0E0F8FF2002F040
:10246000DDF8002002F0DAF8C22002F0E3F80A20DA
:1024700002F0D4F8002002F0D1F8042002F0CEF8E7
:10248000002002F0CBF8C32002F0D4F83C2002F088
:10249000C5F8002002F0C2F83A2002F0BFF8002090
:1024A00002F0BCF8392002F0B9F8002002F0B6F8CA
:1024B000372002F0B3F8002002F0B0F83C2002F020
:1024C000ADF8002002F0AAF8362002F0A7F80020AC
:1024D00002F0A4F8322002F0A1F8002002F09EF8E9
:1024E0002F2002F09BF8002002F098F82C2002F038
:1024F00095F8002002F092F8292002F08FF80020D1
:1025000002F08CF8262002F089F8002002F086F80C
:10251000242002F083F8002002F080F8242002F04A
:102520007DF8002002F07AF8232002F077F80020EE
:1025300002F074F83C2002F071F8002002F06EF80E
:10254000362002F06BF8002002F068F8322002F02A
:1025500065F8002002F062F82F2002F05FF80020FA
:1025600002F05CF82C2002F059F8002002F056F836
:10257000292002F053F8002002F050F8262002F043
:102580004DF8002002F04AF8242002F047F800201D
:1025900002F044F8242002F041F8002002F03EF856
:1025A000232002F03BF8002002F038F8C42002F0AB
:1025B00041F8622002F032F8002002F02FF80520E6
:1025C00002F02CF8002002F029F8842002F026F80E
:1025D000002002F023F8F02002F020F8002002F0A2
:1025E0001DF8182002F01AF8002002F017F8A420B5
:1025F00002F014F8002002F011F8182002F00EF892
:10260000002002F00BF8502002F008F8002002F041
:1026100005F80C2002F002F8002001F0FFFF17205F
:1026200001F0FCFF002001F0F9FF952001F0F6FF1A
:10263000002001F0F3FFF32001F0F0FF002001F093
:10264000EDFFE62001F0EAFF002001F0E7FFC520E2
:1026500001F0F0FF322001F0E1FF002001F0DEFF89
:10266000442001F0DBFF002001F0D8FF652001F0DD
:10267000D5FF002001F0D2FF762001F0CFFF00202F
:1026800001F0CCFF882001F0C9FF002001F0C6FF57
:10269000C62001F0CFFF202001F0C0FF002001F094
:1026A000BDFF172001F0BAFF002001F0B7FF0120A5
:1026B00001F0B4FF002001F0B1FFC72001F0BAFF24
:1026C000002001F0ABFF002001F0A8FF002001F086
:1026D000A5FF002001F0A2FFC82001F0ABFF002001
:1026E00001F09CFF002001F099FF002001F096FF0F
:1026F000002001F093FFC92001F09CFF002001F0B1
:102700008DFF002001F08AFF002001F087FF0020EC
:1027100001F084FF002001F081FF002001F07EFF26
:10272000002001F07BFF002001F078FF002001F085
:1027300075FF002001F072FF002001F06FFF002004
:1027400001F06CFF002001F069FF002001F066FF3E
:10275000002001F063FF002001F060FFE02001F0A5
:1027600069FF162001F05AFF002001F057FF1C20DE
:1027700001F054FF002001F051FF212001F04EFF35
:10278000002001F04BFF362001F048FF002001F04F
:1027900045FF462001F042FF002001F03FFF52209C
:1027A00001F03CFF002001F039FF642001F036FF0A
:1027B000002001F033FF7A2001F030FF002001F00B
:1027C0002DFF8B2001F02AFF002001F027FF992028
:1027D00001F024FF002001F021FFA82001F01EFFDE
:1027E000002001F01BFFB92001F018FF002001F0CC
:1027F00015FFC42001F012FF002001F00FFFCA20D6
:1028000001F00CFF002001F009FFD22001F006FFCB
:10281000002001F003FFD92001F000FF002001F0AB
:10282000FDFEE02001F0FAFE002001F0F7FEF320AB
:1028300001F0F4FE002001F0F1FEE12001F0FAFECB
:10284000162001F0EBFE002001F0E8FE1C2001F054
:10285000E5FE002001F0E2FE222001F0DFFE002074
:1028600001F0DCFE362001F0D9FE002001F0D6FE9A
:10287000452001F0D3FE002001F0D0FE522001F0EF
:10288000CDFE002001F0CAFE642001F0C7FE00204A
:1028900001F0C4FE7A2001F0C1FE002001F0BEFE6E
:1028A0008B2001F0BBFE002001F0B8FE992001F062
:1028B000B5FE002001F0B2FEA82001F0AFFE00201E
:1028C00001F0ACFEB92001F0A9FE002001F0A6FE47
:1028D000C42001F0A3FE002001F0A0FECA2001F0F8
:1028E0009DFE002001F09AFED22001F097FE00200C
:1028F00001F094FED82001F091FE002001F08EFE40
:10290000E02001F08BFE002000E08BE301F086FE6A
:10291000F32001F083FE002001F080FEE22001F0B0
:1029200089FE052001F07AFE002001F077FE0B20E1
:1029300001F074FE002001F071FE1B2001F06EFE1C
:10294000002001F06BFE342001F068FE002001F051
:1029500065FE442001F062FE002001F05FFE4F2082
:1029600001F05CFE002001F059FE612001F056FEEE
:10297000002001F053FE792001F050FE002001F00C
:102980004DFE882001F04AFE002001F047FE97200E
:1029900001F044FE002001F041FEA62001F03EFEC1
:1029A000002001F03BFEB72001F038FE002001F0CE
:1029B00035FEC22001F032FE002001F02FFEC720BC
:1029C00001F02CFE002001F029FED12001F026FEAE
:1029D000002001F023FED62001F020FE002001F0AF
:1029E0001DFEDD2001F01AFE002001F017FEF3208D
:1029F00001F014FE002001F011FEE32001F01AFEA8
:102A0000052001F00BFE002001F008FE0A2000E086
:102A100006E301F003FE002001F000FE1C2001F09F
:102A2000FDFD002001F0FAFD332001F0F7FD00204C
:102A300001F0F4FD442001F0F1FD002001F0EEFD75
:102A4000502001F0EBFD002001F0E8FD622001F0D4
:102A5000E5FD002001F0E2FD782001F0DFFD00201F
:102A600001F0DCFD882001F0D9FD002001F0D6FD49
:102A7000972001F0D3FD002001F0D0FDA62001F049
:102A8000CDFD002001F0CAFDB72001F0C7FD0020F8
:102A900001F0C4FDC22001F0C1FD002001F0BEFD27
:102AA000C72001F0BBFD002001F0B8FDD12001F0EE
:102AB000B5FD002001F0B2FDD52001F0AFFD0020F2
:102AC00001F0ACFDDD2001F0A9FD002001F0A6FD24
:102AD000F32001F0A3FD002001F0A0FDE42001F0AF
:102AE000A9FD012001F09AFD002001F097FD0120D1
:102AF00001F094FD002001F091FD022001F08EFD17
:102B0000002001F08BFD2A2001F088FD002001F05B
:102B100085FD3C2001F082FD002001F07FFD4B206F
:102B200001F07CFD002001F079FD5D2001F076FDD3
:102B3000002001F073FD742001F070FD002001F011
:102B40006DFD842001F06AFD002001F067FD9320F7
:102B500001F064FD002001F061FDA22001F05EFDA6
:102B6000002001F05BFDB32001F058FD002001F0D2
:102B700055FDBE2001F052FD002001F04FFDC420A4
:102B800001F04CFD002001F049FDCD2001F046FD93
:102B9000002001F043FDD32001F040FD002001F0B2
:102BA0003DFDDD2001F03AFD002001F037FDF3206E
:102BB00001F034FD002001F031FDE52001F03AFD87
:102BC000002001F02BFD002001F028FD002001F085
:102BD00025FD002001F022FD022001F01FFD002054
:102BE00001F01CFD292001F019FD002001F016FD67
:102BF0003C2001F013FD002001F010FD4B2001F0FE
:102C00000DFD002001F00AFD5D2001F007FD002010
:102C100001F004FD742001F001FD002001F0FEFC34
:102C2000842001F0FBFC002001F0F8FC932001F06F
:102C3000F5FC002001F0F2FCA22001F0EFFC0020E6
:102C400001F0ECFCB32001F0E9FC002001F0E6FC0F
:102C5000BE2001F0E3FC002001F0E0FCC42001F004
:102C6000DDFC002001F0DAFCCD2001F0D7FC0020D3
:102C700001F0D4FCD32001F0D1FC002001F0CEFC07
:102C8000DC2001F0CBFC002001F0C8FCF32001F0B7
:102C9000C5FC002001F0C2FCE62001F0CBFC1120B5
:102CA00001F0BCFC002001F0B9FC342001F0B6FCBE
:102CB000002001F0B3FC562001F0B0FC002001F030
:102CC000ADFC762001F0AAFC002001F0A7FC7720E3
:102CD00001F0A4FC002001F0A1FC662001F09EFCA4
:102CE000002001F09BFC882001F098FC002001F0FE
:102CF00095FC992001F092FC002001F08FFCBB2094
:102D000001F08CFC002001F089FC992001F086FC88
:102D1000002001F083FC662001F080FC002001F01F
:102D20007DFC552001F07AFC002001F077FC552055
:102D300001F074FC002001F071FC452001F06EFCF4
:102D4000002001F06BFC432001F068FC002001F042
:102D500065FC442001F062FC002001F05FFCE720EC
:102D600001F068FC322001F059FC002001F056FC13
:102D7000552001F053FC002001F050FC762001F0BA
:102D80004DFC002001F04AFC662001F047FC0020C9
:102D900001F044FC672001F041FC002001F03EFC02
:102DA000672001F03BFC002001F038FC872001F097
:102DB00035FC002001F032FC992001F02FFC0020AE
:102DC00001F02CFCBB2001F029FC002001F026FCC6
:102DD000992001F023FC002001F020FC772001F075
:102DE0001DFC002001F01AFC442001F017FC00201B
:102DF00001F014FC562001F011FC002001F00EFC43
:102E0000232001F00BFC002001F008FC332001F02E
:102E100005FC002001F002FC452001F0FFFB002032
:102E200001F0FCFBE82001F005FC002001F0F6FBBE
:102E3000002001F0F3FB992001F0F0FB002001F0ED
:102E4000EDFB872001F0EAFB002001F0E7FB882082
:102E500001F0E4FB002001F0E1FB772001F0DEFB54
:102E6000002001F0DBFB662001F0D8FB002001F020
:102E7000D5FB882001F0D2FB002001F0CFFBAA2077
:102E800001F0CCFB002001F0C9FBBB2001F0C6FB28
:102E9000002001F0C3FB992001F0C0FB002001F0ED
:102EA000BDFB662001F0BAFB002001F0B7FB552006
:102EB00001F0B4FB002001F0B1FB552001F0AEFBA6
:102EC000002001F0ABFB442001F0A8FB002001F042
:102ED000A5FB442001F0A2FB002001F09FFB552040
:102EE00001F09CFB002001F099FBE92001F0A2FB1E
:102EF000AA2001F093FB002001F090FB002001F0DC
:102F00008DFB002001F08AFB002001F093FBAA203A
:102F100001F084FBCF2001F08DFB002001F07EFB4F
:102F2000002001F07BFB002001F078FB002001F085
:102F300075FB002001F072FB002001F06FFB002008
:102F400001F06CFB002001F069FB002001F066FB42
:102F5000002001F063FB002001F060FB002001F085
:102F60005DFB002001F05AFB002001F057FB002020
:102F700001F054FB002001F051FB002001F04EFB5A
:102F8000F02001F057FB002001F048FB502001F039
:102F900045FB002001F042FB002001F03FFB002038
:102FA00001F03CFBF32001F045FB002001F036FB73
:102FB000F92001F03FFB062001F030FB102001F06A
:102FC0002DFB292001F02AFB002001F027FB3A20ED
:102FD00001F030FB552001F021FB112001F02AFB0C
:102FE0006420FDF757F9292001F024FB352001F07A
:102FF00021FB002001F012FB512001F01BFBFF2000
:1030000001F00CFB532001F015FB2C2001F006FB16
:10301000552001F00FFB822001F000FB2C20FDE386
:10302000A0427DD14FF470435521184601F018FBA2
:103030004FF2010BAA21584601F012FB52214FF228
:10304000020001F00DFB08214FF2030001F008FB24
:1030500001214FF2040001F003FB0D214FF4304039
:1030600001F0FEFA0D214BF2010001F0F9FA0D21F9
:103070004BF2020001F0F4FA34214FF4364001F033
:10308000EFFA34214BF2016001F0EAFA34214BF2FD
:10309000026001F0E5FA0D214FF4314001F0E0FA51
:1030A0000D214BF2011001F0DBFA0D214BF2021061
:1030B00001F0D6FA34214FF4374001F0D1FA34212F
:1030C0004BF2017001F0CCFA34214BF2027001F0A6
:1030D000C7FA00214FF4324001F0C2FA00214BF24E
:1030E000012001F0BDFA00214BF2022001F0B8FAF4
:1030F00024214FF4384001F0B3FA24214BF60100AB
:1031000001F0AEFA24214BF6020001F0A9FA0121E8
:103110004FF43F4001F0A4FA0F214FF4334000E098
:10312000FEE301F09DFA0F214BF2013001F098FA15
:103130000F214BF2023001F093FA34214FF4394061
:1031400001F08EFA34214BF6011001F089FA342196
:103150004BF6021001F084FA08214FF4354001F0DB
:103160007FFA08214BF2015001F07AFA08214BF264
:10317000025001F075FA03214FF4424001F070FA59
:1031800024214FF43A4001F06BFA24214BF6012040
:1031900001F066FA24214BF6022001F061FA0021C9
:1031A0004FF43C4001F05CFA78214BF6014001F00D
:1031B00057FA00214BF6024001F052FA00214FF479
:1031C0003D4001F04DFA78214BF6015001F048FAEC
:1031D00000214BF6025001F043FA00214FF43E402B
:1031E00001F03EFA64214BF6016001F039FA00214A
:1031F0004FF4514001F034FA33214DF2011001F047
:103200002FFA00214DF2021001F02AFA34214DF27A
:10321000031001F025FA00214DF2041001F020FA0C
:103220003A214DF2051001F01BFA00214DF2061073
:1032300001F016FA4A214DF2071001F011FA0021AF
:103240004DF2081001F00CFA5C214DF2091001F06A
:1032500007FA00214DF20A1001F002FA81214DF225
:103260000B1001F0FDF900214DF20C1001F0F8F9FE
:10327000A6214DF20D1001F0F3F900214DF20E10D0
:1032800001F0EEF9E5214DF20F1001F0E9F901210D
:103290004DF2101001F0E4F913214DF2111001F07C
:1032A000DFF901214DF2121001F0DAF954214DF24B
:1032B000131001F0D5F901214DF2141001F0D0F9ED
:1032C00082214DF2151001F0CBF901214DF21610BB
:1032D00001F0C6F9CA214DF2171001F0C1F902211F
:1032E0004DF2181001F0BCF900214DF2191001F057
:1032F000B7F902214DF21A1001F0B2F901214DF295
:103300001B1001F0ADF902214DF21C1001F0A8F9DB
:1033100034214DF21D1001F0A3F902214DF21E10CF
:1033200001F09EF967214DF21F1001F099F9022179
:103330004DF2201001F094F984214DF2211001F09A
:103340008FF902214DF2221001F08AF9A4214DF2E9
:10335000231001F085F902214DF2241001F080F9CB
:10336000B7214DF2251001F07BF902214DF2261014
:1033700001F076F9CF214DF2271001F071F9022109
:103380004DF2281001F06CF9DE214DF2291001F008
:1033900067F902214DF22A1001F062F9F2214DF293
:1033A0002B1001F05DF902214DF22C1001F058F9BB
:1033B000FE214DF22D1001F053F903214DF22E1094
:1033C00001F04EF910214DF22F1001F049F90321BF
:1033D0004DF2301001F044F933214DF2311001F07B
:1033E0003FF903214DF2321001F03AF96D214DF20F
:1033F000331001F035F900214FF4524001F030F95B
:1034000033214DF2012001F02BF900214DF2022071
:1034100001F026F934214DF2032001F021F90021B9
:103420004DF2042001F01CF93A214DF2052001F083
:1034300017F900214DF2062001F012F94A214DF250
:10344000072001F00DF900214DF2082001F008F9E4
:103450005C214DF2092001F003F900214DF20A2010
:1034600001F0FEF881214DF20B2001F0F9F8002166
:103470004DF20C2001F0F4F8A6214DF20D2001F0E0
:10348000EFF800214DF20E2001F0EAF8E5214DF2AF
:103490000F2001F0E5F801214DF2102001F0E0F8D5
:1034A00013214DF2112001F0DBF801214DF2122021
:1034B00001F0D6F854214DF2132001F0D1F801218A
:1034C0004DF2142001F0CCF882214DF2152001F0CC
:1034D000C7F801214DF2162001F0C2F8CA214DF2C1
:1034E000172001F0BDF802214DF2182001F0B8F8C4
:1034F00000214DF2192001F0B3F802214DF21A20FB
:1035000001F0AEF801214DF21B2001F0A9F80221D3
:103510004DF21C2001F0A4F834214DF21D2001F0E1
:103520009FF802214DF21E2001F09AF867214DF21A
:103530001F2001F095F802214DF2202001F090F8B3
:1035400084214DF2212001F08BF802214DF222203E
:1035500001F086F8A4214DF2232001F081F8022128
:103560004DF2242001F07CF8B7214DF2252001F026
:1035700077F802214DF2262001F072F8CF214DF2AA
:10358000272001F06DF802214DF2282001F068F8A3
:10359000DE214DF2292001F063F802214DF22A20AC
:1035A00001F05EF8F2214DF22B2001F059F80221D2
:1035B0004DF22C2001F054F8FE214DF22D2001F0A7
:1035C0004FF803214DF22E2001F04AF810214DF260
:1035D0002F2001F045F803214DF2302001F040F892
:1035E00033214DF2312001F03BF803214DF232201E
:1035F00001F036F86D214DF2332001F031F8002151
:103600004FF4534001F02CF833214DF2013001F01A
:1036100027F800214DF2023001F022F834214DF25A
:10362000033001F01DF800214DF2043001F018F8CC
:103630003A214DF2053001F013F800214DF2063029
:1036400001F00EF84A214DF2073001F009F800218F
:103650004DF2083001F004F85C214DF2093000F021
:10366000FFFF00214DF20A3000F0FAFF81214DF2F8
:103670000B3000F0F5FF00214DF20C3000F0F0FFB0
:10368000A6214DF20D3000F0EBFF00214DF20E307F
:1036900000F0E6FFE5214DF20F3000F0E1FF0121DF
:1036A0004DF2103000F0DCFF13214DF2113000F02C
:1036B000D7FF01214DF2123000F0D2FF54214DF21C
:1036C000133000F0CDFF01214DF2143000F0C8FF9F
:1036D00082214DF2153000F0C3FF01214DF216306A
:1036E00000F0BEFFCA214DF2173000F0B9FF0221F1
:1036F0004DF2183000F0B4FF00214DF2193000F007
:10370000AFFF02214DF21A3000F0AAFF01214DF265
:103710001B3000F0A5FF02214DF21C3000F0A0FF8D
:1037200034214DF21D3000F09BFF02214DF21E307E
:1037300000F096FF67214DF21F3000F091FF02214B
:103740004DF2203000F08CFF84214DF2213000F04A
:1037500087FF02214DF2223000F082FFA4214DF2BA
:10376000233000F07DFF02214DF2243000F078FF7D
:10377000B7214DF2253000F073FF02214DF22630C3
:1037800000F06EFFCF214DF2273000F069FF0221DB
:103790004DF2283000F064FFDE214DF2293000F0B8
:1037A0005FFF02214DF22A3000F05AFFF2214DF264
:1037B0002B3000F055FF02214DF22C3000F050FF6D
:1037C000FE214DF22D3000F04BFF03214DF22E3043
:1037D00000F046FF10214DF22F3000F041FF032191
:1037E0004DF2303000F03CFF33214DF2313000F02B
:1037F00037FF03214DF2323000F032FF6D214DF2E0
:10380000333000F02DFF00214FF4544000F028FF2A
:1038100033214DF2014000F023FF00E082E300215C
:103820004DF2024000F01CFF34214DF2034000F045
:1038300017FF00214DF2044000F012FF3A214DF233
:10384000054000F00DFF00214DF2064000F008FF9A
:103850004A214DF2074000F003FF00214DF20840DD
:1038600000F0FEFE5C214DF2094000F0F9FE00215F
:103870004DF20A4000F0F4FE81214DF20B4000F0C1
:10388000EFFE00214DF20C4000F0EAFEA6214DF2C1
:103890000D4000F0E5FE00214DF20E4000F0E0FE8C
:1038A000E5214DF20F4000F0DBFE01214DF210400A
:1038B00000F0D6FE13214DF2114000F0D1FE01219F
:1038C0004DF2124000F0CCFE54214DF2134000F0B6
:1038D000C7FE01214DF2144000F0C2FE82214DF2DC
:1038E000154000F0BDFE01214DF2164000F0B8FE7B
:1038F000CA214DF2174000F0B3FE02214DF21840EC
:1039000000F0AEFE00214DF2194000F0A9FE0221A8
:103910004DF21A4000F0A4FE01214DF21B4000E0E0
:1039200003E300F09DFE02214DF21C4000F098FEE2
:1039300034214DF21D4000F093FE02214DF21E4055
:1039400000F08EFE67214DF21F4000F089FE02213B
:103950004DF2204000F084FE84214DF2214000F021
:103960007FFE02214DF2224000F07AFEA4214DF2AA
:10397000234000F075FE02214DF2244000F070FE5D
:10398000B7214DF2254000F06BFE02214DF226409A
:1039900000F066FECF214DF2274000F061FE0221CB
:1039A0004DF2284000F05CFEDE214DF2294000F08F
:1039B00057FE02214DF22A4000F052FEF2214DF254
:1039C0002B4000F04DFE02214DF22C4000F048FE4D
:1039D000FE214DF22D4000F043FE03214DF22E401A
:1039E00000F03EFE10214DF22F4000F039FE032181
:1039F0004DF2304000F034FE33214DF2314000F002
:103A00002FFE03214DF2324000F02AFE6D214DF2CF
:103A1000334000F025FE00214FF4554000F020FE19
:103A200033214DF2015000F01BFE00214DF20250F7
:103A300000F016FE34214DF2035000F011FE00217B
:103A40004DF2045000F00CFE3A214DF2055000F00A
:103A500007FE00214DF2065000F002FE4A214DF211
:103A6000075000F0FDFD00214DF2085000F0F8FD78
:103A70005C214DF2095000F0F3FD00214DF20A5097
:103A800000F0EEFD81214DF20B5000F0E9FD002128
:103A90004DF20C5000F0E4FDA6214DF20D5000F067
:103AA000DFFD00214DF20E5000F0DAFDE5214DF270
:103AB0000F5000F0D5FD01214DF2105000F0D0FD67
:103AC00013214DF2115000F0CBFD01214DF21250A7
:103AD00000F0C6FD54214DF2135000F0C1FD01214C
:103AE0004DF2145000F0BCFD82214DF2155000F053
:103AF000B7FD01214DF2165000F0B2FDCA214DF282
:103B0000175000F0ADFD02214DF2185000F0A8FD55
:103B100000214DF2195000F0A3FD02214DF21A5080
:103B200000F09EFD01214DF21B5000F099FD022195
:103B30004DF21C5000F094FD34214DF21D5000F068
:103B40008FFD02214DF21E5000F08AFD67214DF2DB
:103B50001F5000F085FD02214DF2205000F080FD45
:103B600084214DF2215000F07BFD02214DF22250C4
:103B700000F076FDA4214DF2235000F071FD0221EA
:103B80004DF2245000F06CFDB7214DF2255000F0AD
:103B900067FD02214DF2265000F062FDCF214DF26B
:103BA000275000F05DFD02214DF2285000F058FD35
:103BB000DE214DF2295000F053FD02214DF22A5032
:103BC00000F04EFDF2214DF22B5000F049FD022194
:103BD0004DF22C5000F044FDFE214DF22D5000F02E
:103BE0003FFD03214DF22E5000F03AFD10214DF221
:103BF0002F5000F035FD03214DF2305000F030FD24
:103C000033214DF2315000F02BFD03214DF23250A3
:103C100000F026FD6D214DF2335000F021FD002112
:103C20004FF4564000F01CFD33214DF2016000F0CE
:103C300017FD00214DF2026000F012FD34214DF21B
:103C4000036000F00DFD00214DF2046000F008FD5E
:103C50003A214DF2056000F003FD00214DF20660AF
:103C600000F0FEFC4A214DF2076000F0F9FC002153
:103C70004DF2086000F0F4FC5C214DF2096000F0A8
:103C8000EFFC00214DF20A6000F0EAFC81214DF2C8
:103C90000B6000F0E5FC00214DF20C6000F0E0FC50
:103CA000A6214DF20D6000F0DBFC00214DF20E600C
:103CB00000F0D6FCE5214DF20F6000F0D1FC0121AF
:103CC0004DF2106000F0CCFC13214DF2116000F0B9
:103CD000C7FC01214DF2126000F0C2FC54214DF2EC
:103CE000136000F0BDFC01214DF2146000F0B8FC3F
:103CF00082214DF2156000F0B3FC01214DF21660F7
:103D000000F0AEFCCA214DF2176000F0A9FC0221C0
:103D10004DF2186000F0A4FC00214DF2196000F093
:103D20009FFC02214DF21A6000F09AFC01214DF235
:103D30001B6000F095FC02214DF21C6000F090FC2D
:103D400034214DF21D6000F08BFC02214DF21E600B
:103D500000F086FC67214DF21F6000F081FC02211B
:103D60004DF2206000F07CFC84214DF2216000F0D7
:103D700077FC02214DF2226000F072FCA4214DF28A
:103D8000236000F06DFC02214DF2246000F068FC1D
:103D9000B7214DF2256000F063FC02214DF2266050
:103DA00000F05EFCCF214DF2276000F059FC0221AB
:103DB0004DF2286000F054FCDE214DF2296000F045
:103DC0004FFC02214DF22A6000F04AFCF2214DF234
:103DD0002B6000F045FC02214DF22C6000F040FC0D
:103DE000FE214DF22D6000F03BFC03214DF22E60D0
:103DF00000F036FC10214DF22F6000F031FC032161
:103E00004DF2306000F02CFC33214DF2316000F0B7
:103E100027FC03214DF2326000F022FC6D214DF2AF
:103E2000336000F01DFC5521184600F019FCAA2152
:103E3000584600F015FC52214FF2020000F010FC31
:103E400008214FF2030000F00BFC00214FF20400A8
:103E500000F006FCCC214FF4314000F001FC0021C1
:103E60004BF2011000F0FCFB05214FF4364000F04E
:103E7000F7FB70214FF4374000F0F2FB70214BF25A
:103E8000017000F0EDFB01214FF4384000F0E8FB39
:103E900003214BF6010000F0E3FB03214BF6020087
:103EA00000F0DEFB03214BF6030000F0D9FB0221FA
:103EB0004FF43C4000F0D4FB00214BF6014000F0F1
:103EC000CFFB00214BF6024000F0CAFBD0214FF49B
:103ED000494000F0C5FB02214CF6011000F0C0FB88
:103EE00050214CF6021000F0BBFB50214CF60310A1
:103EF00000F0B6FB50214CF6041000F0B1FB00219D
:103F00004FF4545000F0ACFB55214FF4685000F0D2
:103F1000A7FB4FF4885000F08DFB7820FCF7BFF929
:103F20004FF4245000F086FBB9E0B842FCD1E22007
:103F300000F080FB1D2000F071FB022000F06EFB02
:103F4000042000F06BFB6420FCF7A9F9E02000F0EE
:103F500071FB012000F062FB0A20FCF79BF9E020D6
:103F600000F068FB032000F059FB0C20FCF792F9ED
:103F7000012000F05FFB0A20FCF78CF9E62000F03E
:103F800059FB2F2000F04AFBFF2000F047FBFF20E9
:103F900000F044FBB02000F04DFB202000F03EFB81
:103FA000002000F03BFB032000F038FB40F21F3004
:103FB00000F034FB012000F031FB40F2DF1000F094
:103FC0002DFB002000F02AFBB42000F033FB04207E
:103FD00000F024FB40F21F4000F020FB002000F026
:103FE0001DFB2E2000F01AFB002000F017FB002024
:103FF00000F014FB002000F011FB002000F00EFB8D
:10400000B62000F017FB022000F008FB4FF403700D
:1040100000F004FB002000F001FB172000F0FEFA86
:10402000152000F0FBFA002000F0F8FA002000F064
:10403000F5FAF02000F0FEFA032000F0EFFA292054
:1040400000F0F8FAD02000F0F5FA002000F0E6FACF
:10405000BE2000F0EFFA052000F0E0FAFE2000F0AC
:10406000DDFA012000F0DAFA002000F0D7FA002093
:1040700000F0D4FA002000F0D1FAB82000F0DAFA0B
:10408000032000F0CBFA012000F0C8FABA2000F0BB
:10409000D1FA012000F0C2FA642000F063F8A88889
:1040A000484505D0B04203D0A04201D0B84209D162
:1040B0000520009002906946D8F82C30D8E901021A
:1040C000FCF722F9A98808A0FBF7A0FF0020FDF764
:1040D00049FD084801222021FCF7E6F85046FDF78B
:1040E0001DFD15B0BDE8F08F4C43442049443A25EE
:1040F000780D0A00000402581FB5FCF7DAF8032215
:1041000001218DF80010500701901B208DF8080048
:1041100000208DF80C008DF809008DF80D008DF849
:104120000A008DF80E0068468DF801208DF80B20EE
:104130008DF80F10FCF7C2F80420FCF7C4F81FBD7F
:104140000346012000E05843491EC9B2FBD2704724
:10415000034808B50088ADF80000BDF8000008BDB0
:10416000000008600246BE2000B500F063FA05209A
:1041700000F054FA00EE102A9FED0D1BB8EE400B34
:1041800020EE010BBCEEC00B10EE100A80B200F066
:1041900045FA012000F042FAFF2000F03FFA00202B
:1041A00000F03CFA5DF804EB002000F037BA0000A4
:1041B0006666666666660440F0B56C4D002341F69F
:1041C00063142946AA798988012A01D01AB11BE013
:1041D000A14202D118E0A14216D1082814D2DFE88A
:1041E00000F00406080A0C0E101206200CE007204E
:1041F0000AE0042008E0052006E0012004E0002099
:1042000002E0032000E0022045F21032A1F513473E
:1042100045F21056413F05D0914203D0B14201D042
:10422000A14277D1082812D2DFE800F01104060875
:104230000A0C0E1080230AE0402308E0C02306E0A9
:10424000202304E0602302E0A02300E0E023B14249
:1042500002D14FF4585000E03620914205D0B142CF
:1042600003D0A14201D043F00803194600F0F8F949
:10427000AA88A2420AD069889806288802D588426E
:1042800002D303E0884201D929806880B24268895C
:1042900041D100F0CFF9002000F0C0F96889401C3E
:1042A00080B200F0C7F9002000F0B8F96889801CDE
:1042B00080B200F0BFF92888401EC0F30F2000F044
:1042C000ADF96889C01C80B200F0B4F92878401EAE
:1042D000C0B200F0A3F9A88900F0ACF9002000F00A
:1042E0009DF9A889401C80B200F0A4F9002000F0DC
:1042F00095F9A889801C80B200F09CF96888401E5E
:10430000C0F30F2000F08AF9A889C01C80B200F029
:1043100091F922E028E000F08DF9002000F07EF90C
:10432000002000F07BF92888401EC0F30F2000F029
:1043300075F92878401EC0B200F070F9A88900F025
:1043400079F9002000F06AF9002000F067F9688828
:10435000401EC0F30F2000F061F9A878BDE8F040DE
:10436000401EC0B200F05AB9F0BD0000C8010024E0
:10437000F0B53F4D060A0C4602462846270AA98892
:104380004089A1F51343413B28D0A1F5A643103B3A
:1043900024D0A1F5C853633B2FD0A1F5AA43103B0D
:1043A00064D100F047F9304600F038F96889401CC4
:1043B00080B200F03FF9D0B200F030F9A88900F0E7
:1043C00039F9384600F02AF9A889401C80B200F07B
:1043D00031F9E0B2BDE8F04000F020B900F02AF970
:1043E000304600F01BF9D0B200F018F9A88900F0AF
:1043F00021F9384600F012F9EBE7A97929B300F06A
:1044000019F9304600F00AF9D0B200F007F928880F
:10441000401EC0F30F2000F001F92878401EC0B202
:1044200000F0FCF8A88900F005F9384600F0F6F82D
:10443000E0B200F0F3F86888401EC0F30F2000F0EF
:10444000EDF8A878401EC0B2C4E72988891A491E31
:104450008AB200F0EFF8002000F0E0F8002000F051
:10446000DDF8100A00F0DAF8D0B2D9E7F0BD0000AC
:10447000C80100242DE9F84F1F460E4682468B46A0
:10448000580700D00120790800EBD700203A10FB34
:1044900001F0002502F0FF09C0B2009047E00C2FA8
:1044A00010D0102F12D0182F14D0202F42D1224913
:1044B00001EBC9104FF00008445D200610D51F48DD
:1044C000026811E01E4909EB490006E01D4901EBB5
:1044D0000910EFE71C4909EBC90001EB8000E9E78F
:1044E0000A9828B91548426831465046FDF7B4FB92
:1044F0006006761C040E1548B6B24088B04219D941
:10450000A6EB0B00B84209D10AF101005E461FFA82
:1045100080FA0E48018851450CD906E008F10100E7
:1045200000F0FF08B8F1080FC7D36D1CEDB200987A
:104530008542B4D3BDE8F88F247000902400002495
:1045400064580090D85C0090C8620090C8010024B4
:104550002DE9FF4F81B01D460027924680463C461C
:10456000DDF838B0B9464FEA5B0627E0281B401E4D
:10457000C1B20A20FFF7E4FDBAFBF0F00A21B0FB5C
:10458000F1F201FB120027B9691E8C4201DA48B131
:1045900001275B463030CDF80090C2B206FB0480A4
:1045A00080B206E006FB048020225B4680B2CDF894
:1045B00000900299FFF75EFF641CE4B2AC42D5D3D1
:1045C00005B0BDE8F08F2DE9F84F00F0FF08044674
:1045D00010190D461FFA80FA4FF0000B58191FFAF8
:1045E00080F9DDE90A7611E0544502D3E819444622
:1045F00085B24D450FD23B4629462046CDF800B046
:10460000FFF738FF04EB570084B2761C3278A2F132
:1046100020005E28E8D9BDE8F88F000001B5BDF89C
:104620000000ADF80000BDF800000149088008BD99
:104630000000086001B5BDF80000ADF80000BDF84D
:1046400000000149088008BDFEFF076002480349D9
:104650000089088070470000C8010024FEFF076041
:10466000024A1080901C018070470000FEFF076026
:10467000104810B586B0016841F002010160006881
:1046800001210D4C00F0020005900320CDE900014E
:10469000CDE9021069462046FBF7DEFD01222046E7
:1046A0001146FBF701FE012220460221FBF7FCFD2B
:1046B00006B010BDE04402580004025808B500904E
:1046C0000548018BC08A491E8BB2401E82B2002170
:1046D000084600F049F808BDB402002400B5AFB0A8
:1046E0004FF000530093CDE9090102200B90CDE972
:1046F0000C026846FCF7E2F9002800D001202FB038
:1047000000BD0000084B10B51C465875A1888AB240
:10471000218889B220B1012801D1D9821A8310BD24
:10472000DA82198310BD0000B4020024F0B50C4FEA
:1047300094B2DFF830C03D467E7D2B68EA692D7D5E
:104740005CF8255026B103FB01004243AC52F0BD9A
:104750007E68301A401E03FB001050432C52F0BDFF
:10476000B40200242C0000242DE9F043254E00243F
:10477000DDF81C90757D0DB1054606E077680D46A5
:10478000B91A1A463B1A491E5B1E3068521B96F82E
:1047900014C0DFF87480871A00FB0150F6697F1E91
:1047A00058F82CC0BFB206FB00C51848066846F48E
:1047B0000006066016484FF440360660022646633F
:1047C0000764066826F001060660C563591A4FF4AF
:1047D0008033491C03EB024211434164C0F8389016
:1047E000016841F001010160420202E0641C944250
:1047F00002D241688907F9D5816841F002018160E0
:10480000BDE8F083B40200242C000024D8440258F0
:10481000001000522DE9FF5F00F0BEF9B84D0123F2
:10482000082704460626A0F5864042384FF4F07269
:104830003AD0A4F5E0404FF0170A84384FF448719D
:1048400040D003204FF08C09A4F5E04CBCF1160CCD
:104850004FF4806B4FF4167E42D0A4F5E048B8F1D7
:1048600018084FF4A06C47D0A4F50048B8F116081A
:1048700045D0A4F58058B8F1180843D04AF2010891
:1048800044454FF4407949D140F25651C5E90019E9
:104890008F21298146212982D521A981688118216A
:1048A000E9811C226882ADE04FF48870C5E90020E0
:1048B0002B8128206B81A8810520EF815822288236
:1048C0006F829FE0C5E900122B812E206B81A881A9
:1048D000D220A5F80EA0288216201822688291E026
:1048E000C5E900BE142129816881A020A5F80C909B
:1048F000E98128820C2055E0C5E900C186E0C5E9C0
:1049000000BE83E0C5E900C1A5F80C900A21298208
:1049100010222981E9816982688173E0A4F5204829
:10492000B8F1020816D0A4F52048B8F103081FD04A
:10493000A4F5204CBCF1040C29D0A4F52040053886
:1049400033D0A4F5204006383ED0A4F520400738E7
:1049500049D05BE0C5E900C12021298130212982AD
:104960005021A9816E810E21E9811622688249E0D9
:10497000C5E900C9202129815021A981302129823E
:10498000072169810C21E981172268823AE0C5E993
:1049900000B98821298118212982A021A9816E814D
:1049A0001D21E981122268822CE04FF45470C5E980
:1049B000000270202881A881102028822F226F8178
:1049C000A5F80EA06E821DE0C5E9001E802028819A
:1049D0005820A8812820288204206881A5F80EA0EC
:1049E00028226B820EE04FF42070C5E9000260209F
:1049F00028812F823820A881022068812921E9811D
:104A00003E226882A0210520FFF768FE3D484FF056
:104A100000082A683D4F3E4B0280696841800220B1
:104A2000E861394838603648A838C0E90038C0F82D
:104A30000880A4F58053C0F80C80183BC0F81080A3
:104A400002D14FF0805303612C89631E43616B894F
:104A5000A3F1010CC0F818C0B5F80CC06444A4F16F
:104A6000010CC0F81CC0B5F80EC06344A3F1010CE2
:104A7000C0F820C0A2F1010CA444C0F824C0A1F1E8
:104A8000010C9C44C0F828C0B5F810C06244224410
:104A9000521EC2626A8A11441944491E016380F899
:104AA000368080F8358080F834801548A838FBF7C8
:104AB000A9FD0720CDE90086CDE902083968FF236A
:104AC0000222002000F028F8A8880022114680B2B7
:104AD0000090288883B2104600F04CF80020FFF7C1
:104AE00011FE0C480122202185F81480FBF7DCFB25
:104AF00004B04FF0FF30BDE8F05FFFF7DFBD00000E
:104B0000B4020024C8010024000000C02C000024CE
:104B100000100050000402582DE9F0438DB01646F5
:104B200014AA134D00240DF1240E92E88013009472
:104B300002942A6801926D68CDE904634FEA082364
:104B40000395CDE906734FEA092308938EE8260002
:104B5000024607488DF8324069468DF83140A83842
:104B60008DF830C0FBF724FD0DB0BDE8F0830000E8
:104B7000B402002470B51E46044603460548049D51
:104B8000FBF71CFE23462A4631460248BDE870402A
:104B9000FBF73EBE0C0200242B4830B587B00168FD
:104BA00041F400710160016801F400710591016830
:104BB00041F48061016000686946244C00F4806023
:104BC0000590402000900020019003200390204693
:104BD000FBF742FB1E4D4420694600902846FBF738
:104BE0003BFB40212046FBF750FB042104462846AE
:104BF000FBF74BFB44EA400428464021FBF745FB0A
:104C000044EA800010F0FF000CD001280DD00228EB
:104C10000ED003280FD0042810D0052811D0002072
:104C200007B030BD44F24230FAE747F28400F7E7BC
:104C300047F21600F4E747F21800F1E748F21600D1
:104C4000EEE741F21800EBE7E04402580024025876
:104C500000280258F0B504688B88E568C5F30B4559
:104C60002B441D04882303EBC213E65806F4704658
:104C7000E65004680F68E668C6F30B46761C3E44AF
:104C80002E43E65003688C89DD68C5F30A052C4481
:104C900025048C2404EBC2141E5906F470461E51E0
:104CA00003688F68DE68C6F30A06761C3E442E430E
:104CB0001E510468942303EBC213E55825F0070541
:104CC000E55005680C69EC5091F8313005681F0219
:104CD00091F832301C040B7E1E069C2303EBC2139A
:104CE00055F803C04FF0000C45F803C091F8305060
:104CF00034433D4325430468E5500468982303EB9F
:104D0000C213E55825F0FF05E55005684C69EC50E5
:104D10000468A02303EBC213E55840F20776B543BD
:104D2000E550D1E907452C430568EC500468AC23F5
:104D300003EBC213E55844F803C005684C6AEC5015
:104D40000B698BB3012B32D0042B32D0022B30D025
:104D5000032B2ED0072B2CD001230568B02404EBA5
:104D6000C2142E5906F0E0262E51D1E90065AD1B84
:104D70000E8D5D435E43ED1D45EA064305682B51EC
:104D80000468B42303EBC213E5586FF30A05E5503A
:104D90000468C96AE1500068842101EBC2114258DD
:104DA00042F001024250F0BDFFE70423D5E70323A0
:104DB000D3E70223D1E77047704700002DE9F047A1
:104DC000DFF8E48004460F464FF00009D8F80000F1
:104DD000C043800709D0344D283D286820F080600A
:104DE0002860FBF748FA064607E00120BDE8F08797
:104DF000FBF741FA801B02284ED828680001F7D43F
:104E0000D8F80010226821F47C3141EA0231C8F858
:104E10000010207A4FF4FE02A1884002491EA0F53E
:104E2000007080B2C1F308010843A189491E02EA5B
:104E300001410843217C1202491E02EA0161084334
:104E40001949103108601848001D0168626921F095
:104E5000C001114301600168A26921F020011143E2
:104E600001606FB10168012F0ED041F400110160A3
:104E7000286840F080602860FBF7FDF904460DE0EB
:104E8000016841F40021F2E741F48011EFE7FBF7FC
:104E9000F2F9001B022801D90320A7E728680001C6
:104EA000F5D54846A2E70000284402582DE9F0470E
:104EB000DFF8E48004460F464FF00009D8F8000000
:104EC000C043800709D0344D283D286820F0805029
:104ED0002860FBF7D0F9064607E00120BDE8F0871F
:104EE000FBF7C9F9801B02284ED828688000F7D448
:104EF000D8F80010228821F07C7141EA0251C8F8EC
:104F00000010207A4FF4FE02A1884002491EA0F54D
:104F1000007080B2C1F308010843A189491E02EA6A
:104F200001410843217C1202491E02EA0161084343
:104F30001949183108601848001D0168626921F498
:104F40004061114301600168A26921F400711143BD
:104F500001606FB10168012F0ED041F080710160D6
:104F6000286840F080502860FBF785F904460DE082
:104F7000016841F48001F2E741F40001EFE7FBF73B
:104F80007AF9001B022801D90320A7E728688000CE
:104F9000F5D54846A2E700002844025808B5034862
:104FA0006946FCF7F9F9009808BD0000D402002416
:104FB00038B50D46044606486946FCF7EDF9009AF7
:104FC000291B491CB2FBF1F001FB1020204438BD25
:104FD000D402002470B5104E00240E4830603046D4
:104FE000FCF7C4F93046FCF70AFA42F2107504E007
:104FF000641CA4B20A20FBF752F930684068C04331
:10500000C00701D0AC42F3D3AC4201D3012070BD44
:10501000002070BD00180248D40200241548012267
:1050200000B5134987B0202301600021C0E90112B7
:105030000822C0E90323402343615301C0E906313C
:10504000130203625302C0E90931062102200090D5
:10505000CDE90121CDE90310059069460690054888
:10506000FCF706FA034800F007F807B000BD00009F
:1050700040410052D8010024002301221846114665
:1050800010B500F021F84FF4FA70FBF708F900238F
:1050900001221846022100F017F8002308221846C2
:1050A000032100F011F8012240F222230421002004
:1050B00000F00AF8BDE81040024840F2A521FCF7D4
:1050C00099BA0000D80100241FB5002410B10128AE
:1050D00002D002E0102400E008240748CDE90223B2
:1050E0004FF6FF72CDE900146946FCF794FA0028E8
:1050F00000D0012004B010BDD80100247047FBF798
:10510000E7B890F83410C90706D001684A68836B85
:1051100022F400321A434A6090F83410890706D509
:1051200001684A68C36B22F480321A434A6090F8DF
:105130003410490706D501684A68036C22F48022BE
:105140001A434A6090F83410090706D501684A6886
:10515000436C22F400421A434A6090F83410C906A6
:1051600006D501688A68836C22F480521A438A60EB
:1051700090F83410890606D501688A68C36C22F459
:1051800000521A438A6090F83410490611D501681C
:105190004A68036D22F480121A434A60016DB1F52A
:1051A000801F06D101684A68436D22F4C0021A4389
:1051B0004A6090F83410090606D501684A68806D87
:1051C00022F4002202434A607047F8B500250446E5
:1051D000C567FBF750F80746206800686FF07E4609
:1051E000000708D500223B464FF4001120460096E8
:1051F00000F0FAFA60B92068006840070AD500227A
:105200003B464FF480012046009600F0EDFA08B1CD
:105210000320F8BD202084F8790084F87A0000206B
:1052200084F87850F8BD10B5806B0021A0F86A10A2
:10523000A0F86210FCF775FA10BD01680A6822F444
:1052400090720A6001688A6822F001028A60202157
:1052500080F87A10704710B5B0F86C2090F87A306A
:105260000168222B05D0088B40F00800088302203B
:1052700010BD898C8368B3F5805F01D103696BB180
:105280001140426E531C43661170B0F86A10491EFB
:105290000904090CA0F86A1007D015E0436E11400C
:1052A0001980416E891C4166EFE701680A6822F4A3
:1052B00090720A6001688A6822F001028A602021E7
:1052C00080F87A10FBF709F8002010BD2DE9F04FA7
:1052D000044600688025FD4B0021D4F810C087B03B
:1052E000A6680F46D4F81C8046EA0C06D4F814C011
:1052F000A26A4CEA080C46EA0C0632430668DFF85C
:10530000D0C306EA0C061643066020684268E668C9
:1053100022F44052324342602268A0699A4201D08E
:10532000266A3043A66AB6F1005F04D1D4E90B6C5B
:1053300046EA0C0630439668DFF898C306EA0C0686
:10534000064396602068C26A666A22F00F02324302
:10535000C262E14E2068E14AB04210D1126802F008
:105360003802182A74D005DCCAB3082A7AD0102A69
:1053700047D179E0202A7BD0282A7CD17AE0D84E08
:10538000B04209D1126802F00702062A73D2DFE8A0
:1053900002F053696B6D6F71D24EB04209D1126841
:1053A00002F00702062A66D2DFE802F0465C5E6081
:1053B0006264CD4EB04209D1126802F00702062A9B
:1053C00059D2DFE802F0394F51535557C74EB0421A
:1053D0000BD1126802F00702062A4CD200E00EE060
:1053E000DFE802F02A4042444648C14EB04209D1AB
:1053F000126802F03802182A38D0BBDCB4E74FF04C
:10540000010538E0BB4EB04209D1126802F0070234
:10541000062A30D2DFE802F01026282A2C2EB64EBB
:10542000B0420BD1126802F00702062A23D2DFE84D
:1054300002F003191B1D1F2100251CE098421AD100
:10544000A64A121D126802F00702062A13D202E0D1
:105450000CE007E00CE0DFE802F0030507090B0DA4
:10546000022508E0042506E0402504E0082502E0C6
:10547000102500E02025DFF864B2A04E9842DFF846
:1054800080A2ABF1540B73D1102D31D006DC022D6C
:1054900009D0042D0AD0082D2FD111E0202D29D0BC
:1054A000402D2AD107E0FBF7F7F913E06846FBF738
:1054B00009FA01980EE003A8FBF782FA049809E0C4
:1054C000DBF800105846890610D50068C0F3C1010A
:1054D0002AFA01F0002811D06168894601EB4101E8
:1054E00081420AD8B0EB093F07D808E05046F3E7FD
:1054F0008448F1E74FF40040EEE7012733E1102D37
:105500004FF000084ED006DC022D0FD0042D15D030
:10551000082D04D12DE0202D4AD0402D13D0012795
:10552000794AA0F54071914270D9E6E7FBF7B4F9EA
:10553000626A0023414636F812200DE06846FBF708
:10554000C1F9019803E003A8FBF73AFA0498002395
:10555000616A36F811201946FAF7C4FE626809023A
:10556000030241EA10615008181841EB080115E0E8
:1055700032E0DBF800105846890609D500680023A0
:10558000C0F3C1012AFA01F0616A36F8112015E072
:10559000606A002336F8102050460FE00023FAF727
:1055A000A1FEBDE7606A002336F81020554805E0EB
:1055B000606A002336F810204FF400400021FAF70B
:1055C00091FE0902020241EA10614FEA59001018E7
:1055D0004A4641EB0801E1E7E3694FF40042934298
:1055E0004DD1082D23D005DC8DB1012D12D0042D15
:1055F00006D112E0102D35D0202D3AD0402D11D0FB
:10560000012721F00F00C1F3420108435AE0FAF7E5
:105610006EFE16E0FAF770FE13E06846FBF752F9EB
:1056200001980EE003A8FBF7CBF9049809E0DBF83A
:1056300000105846890608D50068C0F3C1012AFA4F
:1056400001F0616A36F8111010E0606A36F8101047
:10565000BAFBF1F04100606801EB5001B1FBF0F0E2
:1056600081B2CEE7606A36F810102648B0FBF1F040
:10567000F0E7606A36F81000B2FBF0F0EAE7082DB8
:105680004AD00ADC0DB3012D43D0042D7FF44DAF79
:105690006846FBF717F9019809E0102D52D0202D2C
:1056A00055D0402DF2D103A8FBF78AF90498616A1E
:1056B00036F81110B0FBF1F1606801EB5001B1FB5D
:1056C000F0F080B22168C8604DE01FE0000C005887
:1056D000F369FFCFFFF4FF1100100140544402585A
:1056E0000044004000480040004C00400050004092
:1056F0000014014000780040007C00404C580090AD
:105700000090D00300093D00FFFC0F00FAF7EFFD09
:10571000CDE7FAF7F1FDCAE7DBF80020594692061B
:105720000AD50968C1F3C1022AFA02F1626A36F8A1
:105730001220B1FBF2F20FE0616A36F81120BAFBD9
:10574000F2F209E0616A36F811200949F1E7616A6D
:1057500036F81110B2FBF1F2616802EB5102B2FBB4
:10576000F1F189B2C16007B03846BDE8F08F0000A2
:1057700000093D0090F87910212901D002207047DE
:10578000B0F8621021B18168B1F5805F13D014E0E8
:1057900001680A68920004D58A6822F400028A60CF
:1057A00003E00A6822F080020A600068016841F0A4
:1057B000400101600CE0016961B1C16D4A1CC26524
:1057C000026809781185B0F86210491EA0F86210CD
:1057D00000207047C16D02680988C1F30801118576
:1057E000C16D891CC165EEE72DE9F0411E461746E3
:1057F00088460446069D1CE0681C1AD025B1FAF7BD
:105800003AFD801BA84214D92068016821F4D071A8
:1058100001602068816821F001018160202084F806
:10582000790084F87A00002084F878000320BDE82D
:10583000F0812068C16938EA010004D00020B84234
:10584000DAD00020F3E70120F9E7FEE701000200CB
:105850000400060008000A000C00100020004000B0
:1058600080000001000000000000000000000000B7
:10587000000000003F400000000000000000300079
:10588000400030004000000009000BC03D000BC08C
:105890003D00090018C024407FE022403180000014
:1058A000180024C01B000D803240018003801C4082
:1058B00027401C80074000401000600000000000EE
:1058C000000000000000000000001F802040402079
:1058D0000000402020401F8000000000090006005A
:1058E0001F80060009000000040004003F8004003F
:1058F0000400000000100060000000000000000034
:105900000400040004000400040000000000004043
:105910000000000000000000002001C00600380068
:10592000400000001F802040204020401F800000D9
:10593000000010403FC000400000000018C021409F
:105940002240244018400000108020402440244081
:105950001B80000002000D0011003FC0014000004C
:105960003C80244024402440238000001F802440A9
:1059700024403440038000003000200027C038005D
:10598000200000001B802440244024401B80000095
:105990001C0022C0224022401F80000000000000A6
:1059A000084000000000000000000000046000004B
:1059B00000000000000004000A00110020804040A8
:1059C000090009000900090009000000000040402A
:1059D000208011000A000400180020002340240049
:1059E000180000001F802040274029401F40000071
:1059F000004007C039000F0001C0004020403FC0F8
:105A0000244024401B8000001F8020402040204074
:105A10003080000020403FC0204020401F80000018
:105A200020403FC024402E4030C0000020403FC0F6
:105A300024402E00300000000F0010802040224043
:105A40003380020020403FC0040004003FC02040DB
:105A5000204020403FC02040204000000060202027
:105A600020203FC02000200020403FC024400B00E9
:105A700030C0204020403FC020400040004000C0D7
:105A80003FC03C0003C03C003FC0000020403FC07E
:105A90000C4023003FC020001F80204020402040B9
:105AA0001F80000020403FC0244024001800000058
:105AB0001F802140214020E01FA0000020403FC067
:105AC0002440260019C0004018C024402440224031
:105AD00031800000300020403FC0204030000000F6
:105AE00020003F80004000403F80200020003E001A
:105AF00001C0070038002000380007C03C0007C084
:105B000038000000204039C0060039C020400000A5
:105B10002000384007C0384020000000304021C03D
:105B20002640384020C00000000000007FE04020F8
:105B300040200000000070000C00038000400000C6
:105B40000000402040207FE0000000000000200016
:105B500040002000000000000010001000100010A5
:105B600000100010000000004000000000000000D5
:105B7000000002800540054003C0004020003FC0F7
:105B800004400440038000000000038004400440FF
:105B90000640000000000380044024403FC0004055
:105BA0000000038005400540034000000000044061
:105BB0001FC0244024402000000002E00550055092
:105BC0000650042020403FC00440040003C00040B1
:105BD0000000044027C0004000000000001000103A
:105BE000041027E00000000020403FC001400700F3
:105BF00004C00440204020403FC00040004000005E
:105C000007C0040007C0040003C00000044007C030
:105C10000440040003C0004000000380044004402E
:105C200003800000041007F00450044003800000CB
:105C3000000003800440045007F00010044007C037
:105C4000024004000400000000000640054005403A
:105C500004C00000000004001F8004400040000059
:105C6000040007800040044007C000400400070013
:105C700004C0018006000400060001C0070001C046
:105C800006000000044006C0010006C004400000F9
:105C90000410071004E00180060004000000044026
:105CA00005C00640044000000000000004007BE046
:105CB00040200000000000000000FFF00000000095
:105CC000000040207BE00400000000004000800055
:105CD0004000200020004000000000000000000004
:105CE00000000000000000000000000000001FCCC9
:105CF000000C000000000000000008003000600000
:105D00000800300060000000022003FC1E2002207A
:105D100003FC1E200220000000000E1811043FFFAB
:105D200010840C78000000000F0010840F3800C0B1
:105D3000077818840078000000780F8410C41124BC
:105D40000E9800E40084000808006800700000005D
:105D5000000000000000000000000000000007E05C
:105D60001818200440020000000040022004181807
:105D700007E00000000000000240024001800FF038
:105D800001800240024000000080008000800FF887
:105D900000800080008000000001000D000E000067
:105DA0000000000000000000000000800080008073
:105DB00000800080008000800000000C000C0000CB
:105DC0000000000000000000000000060018006055
:105DD0000180060018002000000007F008081004E9
:105DE0001004080807F000000000080408041FFC65
:105DF000000400040000000000000E0C1014102429
:105E0000104411840E0C000000000C181004110442
:105E1000110412880C700000000000E0032004242C
:105E200008241FFC0024000000001F9810841104A7
:105E30001104108810700000000007F00888110499
:105E4000110418880070000000001C00100010FCF5
:105E500013001C001000000000000E3811441084D4
:105E6000108411440E38000000000700088C104414
:105E70001044088807F00000000000000000030C38
:105E8000030C0000000000000000000000010106FB
:105E9000000000000000000000000080014002201F
:105EA0000410080810040000022002200220022032
:105EB0000220022002200000000010040808041044
:105EC000022001400080000000000E001200100CB3
:105ED000106C10800F00000003E00C1813E4142471
:105EE00017C4082807D000000004003C03C41C406D
:105EF000074000E4001C000410041FFC11041104FE
:105F000011040E880070000003E00C181004100447
:105F1000100410081C10000010041FFC10041004D2
:105F20001004080807F0000010041FFC11041104FD
:105F300017C410040818000010041FFC11041100FD
:105F400017C010000800000003E00C181004100433
:105F500010441C780040000010041FFC10840080D6
:105F6000008010841FFC10040000100410041FFCAB
:105F700010041004000000000003000110011001D3
:105F80001FFE10001000000010041FFC110403800D
:105F90001464181C1004000010041FFC10040004FA
:105FA00000040004000C000010041FFC1F0000FC93
:105FB0001F001FFC1004000010041FFC0C04030051
:105FC00000E010181FFC100007F00808100410046F
:105FD0001004080807F0000010041FFC1084108053
:105FE000108010800F00000007F008181024102403
:105FF000101C080A07F2000010041FFC1104110015
:1060000011C011300E0C000400000E1C110410848D
:10601000108410441C3800001800100010041FFCED
:10602000100410001800000010001FF810040004F5
:10603000000410041FF8100010001E0011E0001CE6
:10604000007013801C0010001FC0103C00E01F00F7
:1060500000E0103C1FC000001004180C163401C0F2
:1060600001C01634180C100410001C00130400FCAE
:1060700013041C00100000000804101C106410849D
:1060800013041C04101800000000000000007FFE34
:106090004002400240020000000030000C0003807B
:1060A0000060001C000300000000400240024002AB
:1060B0007FFE000000000000000000002000400003
:1060C000400040002000000000010001000100012C
:1060D000000100010001000100004000400020001C
:1060E00000000000000000000000009801240144AE
:1060F0000144014400FC000410001FFC008801045E
:106100000104008800700000000000700088010495
:1061100001040104008800000000007000880104F0
:10612000010411081FFC0004000000F801440144B0
:106130000144014400C800000000010401040FFCF8
:106140001104110411001800000000D601290129D2
:10615000012901C90106000010041FFC0084010090
:106160000100010400FC000400000104190419FCF2
:106170000004000400000000000000030001010111
:10618000190119FE0000000010041FFC002400404B
:1061900001B4010C010400000000100410041FFCF5
:1061A0000004000400000000010401FC01040100DF
:1061B00001FC0104010000FC010401FC0084010059
:1061C0000100010400FC0004000000F801040104C7
:1061D0000104010400F80000010101FF0085010431
:1061E00001040088007000000000007000880104B5
:1061F0000104010501FF00010104010401FC008408
:106200000104010001800000000000CC01240124F1
:10621000012401240198000000000100010007F89A
:106220000104010400000000010001F80004000462
:106230000004010801FC0004010001800170000C51
:10624000001001600180010001F0010C003001C06C
:106250000030010C01F0010000000104018C007409
:106260000170018C01040000010101810171000E27
:10627000001801600180010000000184010C01345C
:1062800001440184010C0000000000000000000037
:1062900001003EFC4002400200000000000000003F
:1062A000FFFF0000000000000000400240023EFC32
:1062B000010000000000000000006000800080007D
:1062C000400040002000200000000000000000000E
:1062D00000000000000000000000000000000000BE
:1062E00000000000000000000000000000000000AE
:1062F00000000000000000000000000F80380FFECA
:10630000380F80380000000000000000000000008E
:106310000000000000000100000600000C00003832
:1063200000003100000600000C00003800003000C2
:10633000000000000000000061800067F807F9809D
:106340000061800061800061800061800067F80763
:10635000F98000618000000000000000000001C022
:10636000E003E0F00630080418081FFFFE040E08E2
:106370000787F00381E000000000000001F0000644
:106380000C00040408060C7001F9C0000E00003B6C
:10639000E000EC18070808040C180003E0000000F7
:1063A0000001E00007F003F818041C0804170807B0
:1063B000E1D003C0E00023B0003C0800200800004A
:1063C0001000000000000001000031000032000059
:1063D0001C000000000000000000000000000000A1
:1063E00000000000000000000000000000000000AD
:1063F00000000000000000007F0001FFC00780F0E7
:106400000C00181000042000020000000000002012
:1064100000021000040C00180780F001FFC0007F8C
:10642000000000000000000000000000000000006C
:10643000000000004200006600006600003C000012
:10644000180003FFC0001800003C00006600006652
:1064500000004200000000000800000800000800E2
:1064600000080000080001FFC0000800000800004C
:106470000800000800000800000000000001000003
:106480003100003200001C0000000000000000008D
:1064900000000000000000000000000000000000FC
:1064A00008000008000008000008000008000008BC
:1064B00000000800000800000800000800000000BC
:1064C0000000000000000000380000380000380024
:1064D00000000000000000000000000000000000BC
:1064E0000000000000000000000600001C0000701A
:1064F000000180000E0000380000C0000700001CF2
:106500000000300000000000000000007F8001FF5C
:10651000E003807006001804000804000806001854
:1065200003807001FFE0007F800000000000000099
:10653000000001000801000801000803FFF807FF40
:10654000F80000080000080000080000000000003B
:1065500000000001C03802C058040098040118046B
:106560000218040418061C1803F81801E0F80000CB
:106570000000000000000001C0E003C0F0040008BB
:1065800004080804080806180803F41801E7F000D6
:1065900001E0000000000000000000000300000D0A
:1065A0000000110000610000810803010807FFF8E6
:1065B0000FFFF800010800010800000000000000C3
:1065C00000E007FCD00608080610080610080610B0
:1065D00008061838060FF00607C00000000000008B
:1065E000000000003F8001FFE0038430020818042F
:1065F0001008041008041008071810030FF0000713
:10660000C000000000000000000003C00007000000
:106610000600000600F80607F806180006E0000766
:10662000000006000000000000000001E1E003F7A8
:10663000F0063410041808041808040C08040C08A8
:1066400006161803F3F001C1E0000000000000008E
:10665000F80003FC300306380402080402080402B0
:10666000080404100308F001FFC0007F00000000D0
:10667000000000000000000000000000000000001A
:106680007038007038007038000000000000000012
:1066900000000000000000000000000000000000FA
:1066A00000000000301A00301C0000000000000054
:1066B00000000000000000000000000000000008D2
:1066C0000000140000220000410000808001004012
:1066D0000200200400100800080000000000000074
:1066E00021000021000021000021000021000021E4
:1066F0000000210000210000210000210000000016
:106700000000000000000800080400100200200142
:1067100000400080800041000022000014000008BA
:106720000000000000000003C00004C000040000DE
:10673000080038080F380808380810000C30000727
:10674000E00003C000000000000000003F8000FFE8
:10675000E0038070020F1006708804C0880483086C
:10676000047F8802C09003012000FE400000080062
:1067700000180001F8003E0801C20007020007E20D
:106780000000FE00001FC80001F8000038000008EB
:1067900004000807FFF807FFF804080804080804C5
:1067A000080804080806180803F41801E7F00001B7
:1067B000E0000000000000003F8001FFE003807067
:1067C0000200180400080400080400080400100671
:1067D00000200780C000000004000807FFF807FF42
:1067E000F80400080400080400080400180200105F
:1067F00003807001FFE0007F8000000004000807B4
:10680000FFF807FFF804080804080804080804084B
:1068100008043E080400080600180100600000009B
:1068200004000807FFF807FFF8040808040800043C
:106830000800040800043E00060000060000018075
:1068400000000000000000003F8001FFE0038070B6
:106850000600180400080402080402080203F007F6
:1068600083F000020000020004000807FFF807FFA1
:10687000F8040808000800000800000800000800EC
:1068800004080807FFF807FFF804000800000000EC
:10689000000004000804000804000807FFF807FFD0
:1068A000F8040008040008040008000000000000CC
:1068B00000000000000600000700000104000104C1
:1068C000000104000307FFFE07FFFC0400000400B2
:1068D0000004000004000807FFF807FFF8040C0894
:1068E000001800003E0004C7800503C80600F80435
:1068F000003804001800000804000807FFF807FF2C
:10690000F804000800000800000800000800000863
:1069100000000800001800006000000004000807E4
:10692000FFF807800807FC00007FC00003F800079D
:10693000C000780007800807FFF807FFF804000888
:1069400004000807FFF807000803C00000E000008B
:106950003800001E000007000001C00400F007FF1F
:10696000F8040000000000007F8001FFE003807059
:10697000060018040008040008060018030030018F
:10698000FFE0007F8000000004000807FFF807FF19
:10699000F8040408040400040400040400040400CF
:1069A000060C0003F80001F00000000000000000E9
:1069B0007F8001FFE00380700600880400880400E7
:1069C000C806003C03003E01FFE6007F8400000093
:1069D00004000807FFF807FFF8040808040800048B
:1069E0000C00040F00040BC00610F003F03801E0A7
:1069F0000800000800000001E0F803F03006301045
:106A0000041808041808040C08040C0802061802EC
:106A100007F00781E000000001800006000004008C
:106A20000004000004000807FFF807FFF80400084E
:106A300004000004000006000001800004000007BC
:106A4000FFE007FFF0040018000008000008000045
:106A50000800000800000804001007FFE004000020
:106A600004000006000007E00007FE00041FE0002D
:106A700001F80000380001E0043E0007C0000600F5
:106A80000004000004000007E00007FFC0041FF836
:106A90000007C007F80007FF80043FF80007C004A4
:106AA000F8000700000400000000000400080600D1
:106AB0001807C07805F1C8003E00001F800463E895
:106AC0000780F80600180400080000000400000613
:106AD000000007800007E008047C08001FF800079A
:106AE000F800180804E00807000006000004000091
:106AF0000000000100080600380400F80403E80460
:106B00000F08047C0805F00807C0080700180400F7
:106B10006000000000000000000000000000000015
:106B20000000003FFFFE20000220000220000220A3
:106B30000002200002000000000000000000080029
:106B40000007000000C0000038000006000001C07F
:106B500000003000000E00000100000000000000F6
:106B6000000020000220000220000220000220007D
:106B7000023FFFFE000000000000000000000000D7
:106B800000000000000000000008000010000030BD
:106B9000000020000030000010000008000000008D
:106BA00000000000000001000001000001000001E1
:106BB00000000100000100000100000100000100D0
:106BC00000010000010000010000000000000000C2
:106BD0000020000020000010000010000000000055
:106BE00000000000000000000000000000000000A5
:106BF00000F00019F8001B180022080026080024E5
:106C000008002410003FF8001FF8000008000018DA
:106C100000000004000007FFF80FFFF00018180044
:106C20001008002008002008003018001FF0000F96
:106C3000C00000000000000007C0001FF000183076
:106C4000002008002008002008003C08001C10005C
:106C500000600000000000000000000007C0001FEE
:106C6000F000381800200800200800200804101048
:106C700007FFF80FFFF00000100000000000000008
:106C800000000007C0001FF0001230002218002290
:106C900008002208003208001E10000E200000002C
:106CA00000000000200000200800200801FFF80379
:106CB000FFF806200804200804200807200003002D
:106CC0000000000000000000000E000E6E001FF328
:106CD0000031B10020B10020B1003191001F13003C
:106CE0002E1E00200E00300000000004000807FFE8
:106CF000F80FFFF800100800200000200000200816
:106D0000003FF8001FF8000008000000000000002D
:106D10000000002008002008002008063FF8063F79
:106D2000F800000800000800000800000000000053
:106D3000000000000000000003000003002001002C
:106D40002001002003063FFE063FFC00000000007B
:106D50000000000000000004000807FFF80FFFF823
:106D6000000188000300002FC00038F80020380020
:106D700020080000080000000000000000000400DF
:106D80000804000804000807FFF80FFFF8000008D7
:106D900000000800000800000000000000200800BB
:106DA0003FF8003FF8001008002000003FF8003FC7
:106DB000F8001008002000003FF8003FF80000082D
:106DC000000000002008003FF8003FF80010080015
:106DD0001000002000002008003FF8001FF800000D
:106DE000080000000000000007C0000FF00018308D
:106DF000003008002008002008003008001830008B
:106E00000FF00007C0000000000000002001003F5C
:106E1000FF003FFF0010110020090020080020089B
:106E2000003038001FF0000FC0000000000000001C
:106E300007C0001FF00038180020080020080020BC
:106E400009001011001FFF003FFF000001000000BB
:106E5000002008002008002008003FF8003FF8004C
:106E60000808001008002008002000003000003052
:106E700000000000000000000000000C78001E1858
:106E80000033080023080021080021880021980011
:106E900030F00038600000000000000020000020FA
:106EA0000000200000FFF003FFF800200800200889
:106EB000002008000030000000000000000000007A
:106EC0002000003FF0007FF80000180000080000DC
:106ED00008002010003FF8007FF0000010000000C4
:106EE000000000002000003000003C00003F800057
:106EF00023F0000078000070002380003C00003088
:106F000000002000002000003C00003FE00023F8CB
:106F10000000E0002700003E00003FE00021F800F4
:106F200001E0003E000020000000000020080020DA
:106F300008003838003E680027800003C8002CF89D
:106F40000038380020180020080000000000000071
:106F50002000003003003C01003F830023EC0000D0
:106F600070002380003C0000200000200000000092
:106F70000000000000000038080020380020F80061
:106F800023E8002F88003E08003808002018000081
:106F90007000000000000000000000000000000081
:106FA0000000000008000014001FF7FC300006205D
:106FB00000020000000000000000000000000000CF
:106FC00000000000000000000000FFFFFF000000C4
:106FD00000000000000000000000000000000000B1
:106FE00000002000023000061FF7FC00140000081B
:106FF0000000000000000000000000000000000091
:107000000000001800006000004000004000002068
:1070100000001000000800000400000400000C0044
:107020000010000000000000000000000000000050
:107030000000000000000000000000000000000050
:107040000000000000000000000000000000000040
:107050000000000000000000000000000000000030
:107060000000000000000000000000000000000020
:107070000000000000000000000000000000000010
:107080000000000000000000000000000000000000
:1070900000000000000000000000000000000000F0
:1070A00000000000000000000000000000000000E0
:1070B00000000000000000000000000007F000C019
:1070C00007FFE1E007F001E0000000C00000000061
:1070D00000000000000000000000000000000000B0
:1070E00000000000000000000000000000000000A0
:1070F0000000000000000000000000000000000090
:10710000000000000000000000000000000000007F
:10711000000000000000000000000000000000006F
:10712000000000000000000000000000002000003F
:1071300001C00000078000001F0000001E000000CA
:107140001C20000001C00000078000001F0000009C
:107150001E0000001C0000000000000000000000F5
:10716000000000000000000000000000000000001F
:10717000000000000000000000000000000000000F
:1071800000000000000000000000000000000000FF
:1071900000000000000000000000000000000000EF
:1071A000000000000000000000180C0000180C0097
:1071B00000180FE0001FFC0003F80C0000180C0082
:1071C00000180C0000180C0000180C0000180FE04C
:1071D000001FFC0003F80C0000180C0000180C0045
:1071E000000000000000000000000000000000009F
:1071F000000000000000000000000000000000008F
:10720000000000000000000000000000000000007E
:10721000000000000000000000000000000000006E
:1072200000000000000000000000000000000780D7
:10723000007807C000FC0640010E00200307002074
:10724000020380200FFFFFFC0201C0200200E0606B
:107250000130704001F03F8000F01F00000000008E
:10726000000000000000000000000000000000001E
:10727000000000000000000000000000000000000E
:1072800000000000000000000000000000000000FE
:1072900000000000000000000000000000000000EE
:1072A0000000000000FE000001FF0000030180005C
:1072B00002008060030181C001FF070000FE18008A
:1072C0000000E0000003BF00000CFFC00071806000
:1072D00001C10020030180600000FFC000003F00EA
:1072E000000000000000000000000000000000009E
:1072F000000000000000000000000000000000008E
:10730000000000000000000000000000000000007D
:10731000000000000000000000000000000000006D
:107320000000000000001F0000007FC000FCC0C083
:1073300001FF80600303E0200202782002061E2085
:1073400003FC074001F00380000103C000011C6042
:107350000001E02000010020000100400000018049
:10736000000000000000000000000000000000001D
:10737000000000000000000000000000000000000D
:1073800000000000000000000000000000000000FD
:1073900000000000000000000000000000000000ED
:1073A0000000000000000000002000001C60000041
:1073B0001C4000001F8000000F00000000000000C3
:1073C00000000000000000000000000000000000BD
:1073D00000000000000000000000000000000000AD
:1073E000000000000000000000000000000000009D
:1073F000000000000000000000000000000000008D
:10740000000000000000000000000000000000007C
:10741000000000000000000000000000000000006C
:10742000000000000000000000000000000000005C
:10743000000000000000000000000000000000004C
:107440000007F800003FFF00007807C001C000E01F
:1074500003000030040000080800000410000002CF
:10746000000000000000000000000000000000001C
:10747000000000000000000000000000000000000C
:1074800000000000000000000000000000000000FC
:1074900000000000000000000000000000000000EC
:1074A00000000000000000001000000208000004BE
:1074B000040000080300003001C000E0007807C0AD
:1074C000003FFF000007F80000000000000000007F
:1074D00000000000000000000000000000000000AC
:1074E000000000000000000000000000000000009C
:1074F000000000000000000000000000000000008C
:10750000000000000000000000000000000000007B
:10751000000000000000000000000000000000006B
:10752000000000000000000000000000000C180037
:10753000000E3800000E3800000630000003600026
:107540000061438000FFFF80006143000003600092
:1075500000063000000E3800000E3800000C180045
:10756000000000000000000000000000000000001B
:10757000000000000000000000000000000000000B
:1075800000000000000000000000000000000000FB
:1075900000000000000000000000000000000000EB
:1075A000000000000000000000000000000080005B
:1075B00000008000000080000000800000008000CB
:1075C00000008000007FFF000000800000008000BD
:1075D00000008000000080000000800000008000AB
:1075E000000000000000000000000000000000009B
:1075F000000000000000000000000000000000008B
:10760000000000000000000000000000000000007A
:10761000000000000000000000000000000000006A
:10762000000000000000000000000001000000E376
:10763000000000E2000000FC0000007800000000F4
:10764000000000000000000000000000000000003A
:10765000000000000000000000000000000000002A
:10766000000000000000000000000000000000001A
:10767000000000000000000000000000000000000A
:1076800000000000000000000000000000000000FA
:1076900000000000000000000000000000000000EA
:1076A00000000000000000000000800000008000DA
:1076B00000008000000080000000800000008000CA
:1076C00000008000000080000000800000008000BA
:1076D00000008000000080000000800000008000AA
:1076E000000000000000000000000000000000009A
:1076F000000000000000000000000000000000008A
:107700000000000000000000000000000000000079
:107710000000000000000000000000000000000069
:10772000000000000000000000000000000000C099
:10773000000001E0000001E0000000C000000000C7
:107740000000000000000000000000000000000039
:107750000000000000000000000000000000000029
:107760000000000000000000000000000000000019
:107770000000000000000000000000000000000009
:1077800000000000000000000000000000000000F9
:1077900000000000000000000000000000000000E9
:1077A00000000000000000000000000C0000003895
:1077B000000000E00000038000000E000000380020
:1077C0000000E00000038000000E00000038000010
:1077D00000E00000038000000E0000001800000020
:1077E0000000000000000000000000000000000099
:1077F0000000000000000000000000000000000089
:107800000000000000000000000000000000000078
:107810000000000000000000000000000000000068
:10782000000000000000000000000000000FF80051
:10783000007FFF0000F00780018000C003000060AF
:10784000020000200200002002000020030000606F
:10785000018000C000E00380007FFF00000FF800FF
:107860000000000000000000000000000000000018
:107870000000000000000000000000000000000008
:1078800000000000000000000000000000000000F8
:1078900000000000000000000000000000000000E8
:1078A00000000000000000000000000000000000D8
:1078B0000080002000800020008000200080006008
:1078C00001FFFFE003FFFFE0000000600000002078
:1078D0000000002000000020000000000000000068
:1078E0000000000000000000000000000000000098
:1078F0000000000000000000000000000000000088
:107900000000000000000000000000000000000077
:107910000000000000000000000000000000000067
:10792000000000000000000000000000007800E0FF
:10793000009801600100026002000460020008601B
:1079400002001060020020600200406003008060BE
:107950000183006001FE00E0007C07800000000061
:107960000000000000000000000000000000000017
:107970000000000000000000000000000000000007
:1079800000000000000000000000000000000000F7
:1079900000000000000000000000000000000000E7
:1079A00000000000000000000000000000F0078060
:1079B00001F007C001000040020000200201002089
:1079C0000201002002010020030380200186804084
:1079D00001FCC0C000787F8000001E000000000095
:1079E0000000000000000000000000000000000097
:1079F0000000000000000000000000000000000087
:107A00000000000000000000000000000000000076
:107A10000000000000000000000000000000000066
:107A20000000000000000000000008000000380016
:107A3000000048000001880000060800000C081043
:107A4000003008100040081001FFFFF003FFFFF0B6
:107A500003FFFFF0000008100000081000000810ED
:107A60000000000000000000000000000000000016
:107A70000000000000000000000000000000000006
:107A800000000000000000000000000000000000F6
:107A900000000000000000000000000000000000E6
:107AA000000000000000000000000000000007804F
:107AB000001F864003E10020030200200304002091
:107AC00003040020030400200304002003060040F8
:107AD000030301C00301FF8003007E0000000000DB
:107AE0000000000000000000000000000000000096
:107AF0000000000000000000000000000000000086
:107B00000000000000000000000000000000000075
:107B10000000000000000000000000000000000065
:107B20000000000000000000000000000007FC0052
:107B3000003FFF000070C380008180C00101006031
:107B400003020020020200200202002002020020A4
:107B50000203004001C180C000C0FF8000007E0021
:107B60000000000000000000000000000000000015
:107B70000000000000000000000000000000000005
:107B800000000000000000000000000000000000F5
:107B900000000000000000000000000000000000E5
:107BA00000000000000000000000000000F00000E5
:107BB00003C000000380000003000000030007E092
:107BC00003003FE00301C0000306000003180000AB
:107BD00003600000038000000300000000000000BC
:107BE0000000000000000000000000000000000095
:107BF0000000000000000000000000000000000085
:107C00000000000000000000000000000000000074
:107C10000000000000000000000000000000000064
:107C2000000000000000000000001F0000783F80FE
:107C300000FC60C0018EC0400307802002030020CA
:107C400002018020020180200201C0200301E040E7
:107C5000018670C000FC3F8000781F00000000001B
:107C60000000000000000000000000000000000014
:107C70000000000000000000000000000000000004
:107C800000000000000000000000000000000000F4
:107C900000000000000000000000000000000000E4
:107CA0000000000000000000003F000000FF81C055
:107CB00001C0C1C00100602002002020020020207D
:107CC0000200202002002060020040C00100C180AC
:107CD00000C18F00007FFE00001FF00000000000C8
:107CE0000000000000000000000000000000000094
:107CF0000000000000000000000000000000000084
:107D00000000000000000000000000000000000073
:107D10000000000000000000000000000000000063
:107D20000000000000000000000000000000000053
:107D3000000000000000000000000000000300C080
:107D4000000781E0000781E0000300C000000000A0
:107D50000000000000000000000000000000000023
:107D60000000000000000000000000000000000013
:107D70000000000000000000000000000000000003
:107D800000000000000000000000000000000000F3
:107D900000000000000000000000000000000000E3
:107DA00000000000000000000000000000000000D3
:107DB0000000000000000000000000000006006657
:107DC0000006007800000000000000000000000035
:107DD00000000000000000000000000000000000A3
:107DE0000000000000000000000000000000000093
:107DF0000000000000000000000000000000000083
:107E00000000000000000000000000000000000072
:107E10000000000000000000000000000000000062
:107E200000000000000000000000000000008000D2
:107E30000001C0000003600000063000000C1800C4
:107E400000180C00003006000060030000C0018034
:107E500001000040020000200400001000000000AB
:107E60000000000000000000000000000000000012
:107E70000000000000000000000000000000000002
:107E800000000000000000000000000000000000F2
:107E900000000000000000000000000000000000E2
:107EA00000000000000000000004100000041000AA
:107EB0000004100000041000000410000004100072
:107EC0000004100000041000000410000004100062
:107ED0000004100000041000000410000004100052
:107EE0000000000000000000000000000000000092
:107EF0000000000000000000000000000000000082
:107F00000000000000000000000000000000000071
:107F10000000000000000000000000000000000061
:107F2000000000000000000000000000040000103D
:107F3000020000200100004000C00180006003003A
:107F40000030060000180C00000C1800000630007D
:107F5000000360000001C00000008000000000007D
:107F60000000000000000000000000000000000011
:107F70000000000000000000000000000000000001
:107F800000000000000000000000000000000000F1
:107F900000000000000000000000000000000000E1
:107FA0000000000000000000000000000078000059
:107FB00001F800000238000002000000040000C0C8
:107FC000040079E0040081E0040100C00403000023
:107FD000020200000306000001FC000000F800009F
:107FE0000000000000000000000000000000000091
:107FF0000000000000000000000000000000000081
:108000000000000000000000000000000000000070
:108010000000000000000000000000000000000060
:108020000000000000000000000FF800003FFE000C
:108030000070078000C000C00101F8400307FC2069
:10804000021E04200230082002203020023FFC20C3
:10805000013F044001800CC000E03180001FC200DD
:108060000000000000000000000000000000000010
:108070000000000000000000000000000000000000
:1080800000000000000000000000000000000000F0
:1080900000000000000000000000000000000000E0
:1080A000000000000000002000000060000003E06D
:1080B00000003E200003E020003E200003E02000FE
:1080C0000380200007FC2000003FE0000003FE20AA
:1080D00000003FE0000001E0000000200000002060
:1080E0000000000000000000000000000000000090
:1080F0000000000000000000000000000000000080
:10810000000000000000000000000000000000006F
:10811000000000000000000000000000000000005F
:10812000000000000000000002000020020000200B
:1081300003FFFFE003FFFFE0020100200201002037
:1081400002010020020100200201002003030020A0
:108150000186806001FCC0C000F87F8000001F0025
:10816000000000000000000000000000000000000F
:1081700000000000000000000000000000000000FF
:1081800000000000000000000000000000000000EF
:1081900000000000000000000000000000000000DF
:1081A00000000000000000000007F800003FFF0092
:1081B0000070078000C000C00100004003000020E4
:1081C0000200002002000020020000200200002027
:1081D00001000040018000C003C0018000300600A3
:1081E000000000000000000000000000000000008F
:1081F000000000000000000000000000000000007F
:10820000000000000000000000000000000000006E
:10821000000000000000000000000000000000005E
:10822000000000000000000002000020020000200A
:1082300003FFFFE003FFFFE0020000200200002038
:108240000200002002000020030000600100004046
:10825000018000C000F00780007FFE00000FF800E2
:10826000000000000000000000000000000000000E
:1082700000000000000000000000000000000000FE
:1082800000000000000000000000000000000000EE
:1082900000000000000000000000000000000000DE
:1082A000000000000000000002000020020000208A
:1082B00003FFFFE003FFFFE00201002002010020B6
:1082C00002010020020100200201002002038020A0
:1082D000020FE0200300006003C000E00060030024
:1082E000000000000000000000000000000000008E
:1082F000000000000000000000000000000000007E
:10830000000000000000000000000000000000006D
:10831000000000000000000000000000000000005D
:108320000000000000000000020000200200002009
:1083300003FFFFE003FFFFE0020100200201002035
:108340000201000002010000020100000201000021
:1083500002038000030FE0000300000003C00000E0
:1083600000600000000000000000000000000000AD
:1083700000000000000000000000000000000000FD
:1083800000000000000000000000000000000000ED
:1083900000000000000000000000000000000000DD
:1083A00000000000000000000007F800003FFE0091
:1083B0000070078001C001C00100004003000020E0
:1083C0000200002002000020020000200100202006
:1083D0000100204003C03F8000303F8000002000AB
:1083E000000020000000000000000000000000006D
:1083F000000000000000000000000000000000007D
:10840000000000000000000000000000000000006C
:10841000000000000000000000000000000000005C
:1084200000000000020000200200002003FFFFE027
:1084300003FFFFE002008020020080200000800097
:1084400000008000000080000200802002008020E8
:1084500003FFFFE003FFFFE0020000200200002016
:10846000000000000000000000000000000000000C
:1084700000000000000000000000000000000000FC
:1084800000000000000000000000000000000000EC
:1084900000000000000000000000000000000000DC
:1084A00000000000000000000000000000000000CC
:1084B0000200002002000020020000200200002034
:1084C00003FFFFE003FFFFE00200002002000020A6
:1084D0000200002002000020000000000000000058
:1084E000000000000000000000000000000000008C
:1084F000000000000000000000000000000000007C
:10850000000000000000000000000000000000006B
:10851000000000000000000000000000000000005B
:1085200000000000000000000000000E0000000F2E
:108530000000000F00000001020000010200000125
:10854000020000030200000603FFFFFC03FFFFF828
:108550000200000002000000020000000200000013
:10856000000000000000000000000000000000000B
:1085700000000000000000000000000000000000FB
:1085800000000000000000000000000000000000EB
:1085900000000000000000000000000000000000DB
:1085A0000000000000000000020000200200002087
:1085B00003FFFFE003FFFFE00200C02002010020F4
:1085C00000078000000FE0000030F80002603E204D
:1085D00003800F20030003E0020000E002000020FF
:1085E000000000200000000000000000000000006B
:1085F000000000000000000000000000000000007B
:10860000000000000000000000000000000000006A
:10861000000000000000000000000000000000005A
:108620000000000000000000020000200200002006
:1086300003FFFFE003FFFFE0020000200200002034
:1086400000000020000000200000002000000020AA
:108650000000002000000060000000E000000300B7
:10866000000000000000000000000000000000000A
:1086700000000000000000000000000000000000FA
:1086800000000000000000000000000000000000EA
:1086900000000000000000000000000000000000DA
:1086A00000000000020000200200002003FFFFE0A5
:1086B00003E0002003FF0020001FF0000001FF8006
:1086C00000000FE000001E000003E000003E00205C
:1086D00003E0002003FFFFE003FFFFE002000020B3
:1086E0000200002000000000000000000000000068
:1086F000000000000000000000000000000000007A
:108700000000000000000000000000000000000069
:108710000000000000000000000000000000000059
:1087200000000000020000200200002003FFFFE024
:108730000380002003F0002000FC0000001F000068
:108740000007C0000001F00000007C0002001F8054
:10875000020007E003FFFFE002000000020000004B
:108760000000000000000000000000000000000009
:1087700000000000000000000000000000000000F9
:1087800000000000000000000000000000000000E9
:1087900000000000000000000000000000000000D9
:1087A0000000000000000000000FF800003FFE0085
:1087B00000F00780018000C001000040020000209E
:1087C0000200002002000020020000200100004002
:1087D000018000C000F00380003FFE00000FF800A1
:1087E0000000000000000000000000000000000089
:1087F0000000000000000000000000000000000079
:108800000000000000000000000000000000000068
:108810000000000000000000000000000000000058
:108820000000000000000000020000200200002004
:1088300003FFFFE003FFFFE0020080200200802032
:108840000200800002008000020080000200800020
:10885000030180000183000000FE0000007C000096
:108860000000000000000000000000000000000008
:1088700000000000000000000000000000000000F8
:1088800000000000000000000000000000000000E8
:1088900000000000000000000000000000000000D8
:1088A0000000000000000000000FF800007FFF0043
:1088B00000F00380018001C0010006400200042096
:1088C0000200042002000620020003E0010000F87C
:1088D0000180005C00E0038C003FFF0C000FFC18DF
:1088E0000000000000000000000000000000000088
:1088F0000000000000000000000000000000000078
:108900000000000000000000000000000000000067
:108910000000000000000000000000000000000057
:108920000000000000000000020000200200002003
:1089300003FFFFE003FFFFE002010020020100202F
:10894000020180000201E0000201FC0003033F80FD
:10895000018607E001FC00E000F800200000002094
:108960000000000000000000000000000000000007
:1089700000000000000000000000000000000000F7
:1089800000000000000000000000000000000000E7
:1089900000000000000000000000000000000000D7
:1089A0000000000000000000000000000078060049
:1089B00000FE01E0018600C0030300400203002026
:1089C00002018020020180200201C0200200C0209C
:1089D0000100E060018070C003E03F8000001F00E4
:1089E0000000000000000000000000000000000087
:1089F0000000000000000000000000000000000077
:108A00000000000000000000000000000000000066
:108A10000000000000000000000000000000000056
:108A20000000000000000000006000000380000063
:108A300003000000020000000200002002000020ED
:108A400003FFFFE003FFFFE0020000200200002020
:108A500002000000020000000380000000E00000AF
:108A60000000000000000000000000000000000006
:108A700000000000000000000000000000000000F6
:108A800000000000000000000000000000000000E6
:108A900000000000000000000000000000000000D6
:108AA00000000000020000000200000003FFFF00C1
:108AB00003FFFFC002000040020000600000002031
:108AC0000000002000000020000000200200004004
:108AD0000200008003FFFF0002000000020000000F
:108AE0000000000000000000000000000000000086
:108AF0000000000000000000000000000000000076
:108B00000000000000000000000000000000000065
:108B10000000000000000000000000000000000055
:108B20000000000000000000020000000200000041
:108B300003C0000003FC0000023FC0000003F80077
:108B400000007F80000007E0000007800000780040
:108B50000203C000023C000003C00000020000004D
:108B60000200000000000000000000000000000003
:108B700000000000000000000000000000000000F5
:108B800000000000000000000000000000000000E5
:108B900000000000000000000000000000000000D5
:108BA000000000000200000003C0000003FF80007E
:108BB000023FFE0002007FE000000F000200F00014
:108BC00003EF000003FF8000020FFE0000003FE003
:108BD00000001F000207E00003F80000030000008F
:108BE0000200000000000000000000000000000083
:108BF0000000000000000000000000000000000075
:108C00000000000000000000000000000000000064
:108C10000000000000000000000000000000000054
:108C20000000000000000000020000200200002000
:108C3000038000E003F0032002FC0C20021F300040
:108C40000007C0000007F00002187C0002601F202F
:108C5000038003E0020000E002000020000000208A
:108C60000000000000000000000000000000000004
:108C700000000000000000000000000000000000F4
:108C800000000000000000000000000000000000E4
:108C900000000000000000000000000000000000D4
:108CA00000000000000000000200000003000000BF
:108CB00003C0000003F80000023E0020020FC020A5
:108CC0000001FFE000007FE000038020021C002084
:108CD000027000000380000002000000020000009B
:108CE0000000000000000000000000000000000084
:108CF0000000000000000000000000000000000074
:108D00000000000000000000000000000000000063
:108D10000000000000000000000000000000000053
:108D2000000000000000000000000020006000E0E3
:108D3000038003E003000FA002003E200200F820A1
:108D40000203E020020F8020023E00200278002073
:108D500003E00060038000E0020003000000000068
:108D60000000000000000000000000000000000003
:108D700000000000000000000000000000000000F3
:108D800000000000000000000000000000000000E3
:108D900000000000000000000000000000000000D3
:108DA00000000000000000000000000000000000C3
:108DB0000000000000000000000000001FFFFFFC9A
:108DC0001000000410000004100000041000000453
:108DD0001000000410000004100000040000000057
:108DE0000000000000000000000000000000000083
:108DF0000000000000000000000000000000000073
:108E00000000000000000000000000000000000062
:108E10000000000000000000000000000000000052
:108E20000000000000000000000000000000000042
:108E30000700000003C0000000780000001E0000D2
:108E40000003C0000000F00000001E0000000780CA
:108E5000000000F00000003C0000000600000000E0
:108E60000000000000000000000000000000000002
:108E700000000000000000000000000000000000F2
:108E800000000000000000000000000000000000E2
:108E900000000000000000000000000000000000D2
:108EA00000000000000000000000000010000004AE
:108EB0001000000410000004100000041000000462
:108EC00010000004100000041FFFFFFC0000000061
:108ED0000000000000000000000000000000000092
:108EE0000000000000000000000000000000000082
:108EF0000000000000000000000000000000000072
:108F00000000000000000000000000000000000061
:108F10000000000000000000000000000000000051
:108F20000000000000000000000000000000000041
:108F30000000000002000000040000000800000023
:108F400018000000100000001800000018000000C9
:108F5000040000000200000000000000000000000B
:108F60000000000000000000000000000000000001
:108F700000000000000000000000000000000000F1
:108F800000000000000000000000000000000000E1
:108F900000000000000000000000000000000000D1
:108FA00000000000000000010000000100000001BE
:108FB00000000001000000010000000100000001AD
:108FC000000000010000000100000001000000019D
:108FD000000000010000000100000001000000018D
:108FE0000000000100000000000000000000000080
:108FF0000000000000000000000000000000000071
:109000000000000000000000000000000000000060
:109010000000000000000000000000000000000050
:109020000000000000000000000000000000000040
:1090300010000000100000001000000018000000E8
:109040000800000004000000000000000000000014
:109050000000000000000000000000000000000010
:109060000000000000000000000000000000000000
:1090700000000000000000000000000000000000F0
:1090800000000000000000000000000000000000E0
:1090900000000000000000000000000000000000D0
:1090A00000000000000000000000038000018FC0ED
:1090B00000038C600006182000041020000410201B
:1090C0000004202000042040000620400003FFC0D0
:1090D0000001FFE00000002000000020000000C0B0
:1090E0000000000000000000000000000000000080
:1090F0000000000000000000000000000000000070
:10910000000000000000000000000000000000005F
:10911000000000000000000000000000000000004F
:10912000000000000000000002000000020000003B
:1091300003FFFFE007FFFFC0000180C000020060E6
:109140000002002000040020000400200004002091
:1091500000060040000300C00001FF800000FE0088
:1091600000000000000000000000000000000000FF
:1091700000000000000000000000000000000000EF
:1091800000000000000000000000000000000000DF
:1091900000000000000000000000000000000000CF
:1091A00000000000000000000000000000007E0041
:1091B0000001FF80000381C0000200400006002083
:1091C000000400200004002000040020000600200D
:1091D0000003C0400001C080000003000000000048
:1091E000000000000000000000000000000000007F
:1091F000000000000000000000000000000000006F
:10920000000000000000000000000000000000005E
:10921000000000000000000000000000000000004E
:1092200000000000000000000000000000007E00C0
:109230000001FF80000380C00006006000040020E1
:10924000000400200004002002040040020200800C
:1092500003FFFFE007FFFFC00000004000000040E8
:1092600000000000000000000000000000000000FE
:1092700000000000000000000000000000000000EE
:1092800000000000000000000000000000000000DE
:1092900000000000000000000000000000000000CE
:1092A00000000000000000000000000000007E0040
:1092B0000001FF80000311C0000210400004106094
:1092C00000041020000410200004102000061020CC
:1092D000000310400001F0C0000071000000000019
:1092E000000000000000000000000000000000007E
:1092F000000000000000000000000000000000006E
:10930000000000000000000000000000000000005D
:10931000000000000000000000000000000000004D
:109320000000000000000000000000000004000039
:10933000000400200004002000040020007FFFE063
:1093400001FFFFE0010400200304002002040020CC
:1093500002040020020400000200000001C000001E
:1093600001C000000000000000000000000000003C
:1093700000000000000000000000000000000000ED
:1093800000000000000000000000000000000000DD
:1093900000000000000000000000000000000000CD
:1093A0000000000000000000000000000000001CA1
:1093B0000000E33E0003FFC200020CC3000404C12E
:1093C000000404C1000404C1000404C100060CC16F
:1093D0000003F8C30005F0620006007E0006003CB2
:1093E000000000000000000000000000000000007D
:1093F000000000000000000000000000000000006D
:10940000000000000000000000000000000000005C
:10941000000000000000000000000000000000004C
:1094200000000000000000000200002002000020F8
:1094300003FFFFE007FFFFE0000100200002002023
:1094400000060000000400000004000000040020EA
:10945000000600200003FFE00001FFE00000002004
:1094600000000020000000000000000000000000DC
:1094700000000000000000000000000000000000EC
:1094800000000000000000000000000000000000DC
:1094900000000000000000000000000000000000CC
:1094A00000000000000000000000000000000000BC
:1094B000000400200004002000040020000400201C
:1094C0000387FFE0038FFFE00380002000000020FF
:1094D000000000200000002000000000000000004C
:1094E000000000000000000000000000000000007C
:1094F000000000000000000000000000000000006C
:10950000000000000000000000000000000000005B
:10951000000000000000000000000000000000004B
:10952000000000000000000000000000000000003B
:10953000000000060000000700000001000000011C
:109540000004000100040001000400030004000600
:109550000387FFFC038FFFF803800000000000007A
:1095600000000000000000000000000000000000FB
:1095700000000000000000000000000000000000EB
:1095800000000000000000000000000000000000DB
:1095900000000000000000000000000000000000CB
:1095A0000000000000000000020000200200002077
:1095B00003FFFFE007FFFFE000000820000010208D
:1095C000000030000000FC0000058E00000707A02E
:1095D000000601E0000400E000040020000000207C
:1095E000000000000000000000000000000000007B
:1095F000000000000000000000000000000000006B
:10960000000000000000000000000000000000005A
:10961000000000000000000000000000000000004A
:10962000000000000000000000000000000000003A
:1096300002000020020000200200002002000020A2
:1096400003FFFFE007FFFFE0000000200000002014
:1096500000000020000000200000000000000000CA
:1096600000000000000000000000000000000000FA
:1096700000000000000000000000000000000000EA
:1096800000000000000000000000000000000000DA
:1096900000000000000000000000000000000000CA
:1096A0000000000000000000000400200007FFE0B0
:1096B000000FFFE000020020000400000004002072
:1096C0000007FFE00003FFE00002002000040000AC
:1096D000000400200007FFE00003FFE0000000207E
:1096E000000000000000000000000000000000007A
:1096F000000000000000000000000000000000006A
:109700000000000000000000000000000000000059
:109710000000000000000000000000000000000049
:1097200000000000000000000004002000040020F1
:109730000007FFE0000FFFE0000100200002002012
:1097400000020000000400000004000000040020EB
:10975000000600200003FFE00001FFE00000002001
:1097600000000020000000000000000000000000D9
:1097700000000000000000000000000000000000E9
:1097800000000000000000000000000000000000D9
:1097900000000000000000000000000000000000C9
:1097A00000000000000000000000000000007E003B
:1097B0000000FF80000381C000020040000600207E
:1097C0000004002000040020000400200006002007
:1097D00000020040000381C00001FF8000007E0005
:1097E0000000000000000000000000000000000079
:1097F0000000000000000000000000000000000069
:109800000000000000000000000000000000000058
:109810000000000000000000000000000000000048
:10982000000000000000000000040001000400012E
:109830000007FFFF000FFFFF000100C10002004111
:109840000004002000040020000400200004002088
:1098500000060040000301C00001FF8000007E0000
:1098600000000000000000000000000000000000F8
:1098700000000000000000000000000000000000E8
:1098800000000000000000000000000000000000D8
:1098900000000000000000000000000000000000C8
:1098A00000000000000000000000000000007E003A
:1098B0000001FF80000380C000020060000400205F
:1098C00000040020000400200004002000020041E9
:1098D000000300C10003FFFF0007FFFF00000001BD
:1098E0000000000100000000000000000000000077
:1098F0000000000000000000000000000000000068
:109900000000000000000000000000000000000057
:109910000000000000000000000000000000000047
:1099200000000000000000000004002000040020EF
:109930000004002000040020000FFFE0000FFFE003
:109940000000C020000100200002002000060020CE
:1099500000040000000400000007000000030000F5
:1099600000000000000000000000000000000000F7
:1099700000000000000000000000000000000000E7
:1099800000000000000000000000000000000000D7
:1099900000000000000000000000000000000000C7
:1099A000000000000000000000000000000003E0D4
:1099B0000001C0E00003E040000630200004302039
:1099C00000041820000418200004182000040C20B3
:1099D00000020C60000307C0000783800000000045
:1099E0000000000000000000000000000000000077
:1099F0000000000000000000000000000000000067
:109A00000000000000000000000000000000000056
:109A10000000000000000000000000000000000046
:109A20000000000000000000000000000004000032
:109A30000004000000040000000C0000001FFF8074
:109A400000FFFFC0000400600004002000040020AC
:109A5000000400200004004000000180000000001D
:109A600000000000000000000000000000000000F6
:109A700000000000000000000000000000000000E6
:109A800000000000000000000000000000000000D6
:109A900000000000000000000000000000000000C6
:109AA00000000000000000000004000000040000AE
:109AB0000007FF80000FFFC00000006000000020D2
:109AC00000000020000000200000002000040040F2
:109AD000000400800007FFE0000FFFC0000000400E
:109AE0000000004000000000000000000000000036
:109AF0000000000000000000000000000000000066
:109B00000000000000000000000000000000000055
:109B10000000000000000000000000000000000045
:109B2000000000000000000000040000000400002D
:109B3000000780000007F0000004FE0000041FC0C2
:109B4000000003E00000038000001C00000460002F
:109B50000007800000060000000400000000000074
:109B600000000000000000000000000000000000F5
:109B700000000000000000000000000000000000E5
:109B800000000000000000000000000000000000D5
:109B900000000000000000000000000000000000C5
:109BA0000000000000040000000600000007C000E4
:109BB0000007FC0000043F80000003E000040F8069
:109BC0000006F0000007F0000007FF8000040FE02F
:109BD0000000038000043C000007C00000060000F5
:109BE0000004000000000000000000000000000071
:109BF0000000000000000000000000000000000065
:109C00000000000000000000000000000000000054
:109C10000000000000000000000000000000000044
:109C200000000000000000000000002000040020F0
:109C300000040060000700E0000783200007E60042
:109C40000004F80000003C0000045E20000587A02E
:109C5000000601E000040060000400200000002075
:109C600000000000000000000000000000000000F4
:109C700000000000000000000000000000000000E4
:109C800000000000000000000000000000000000D4
:109C900000000000000000000000000000000000C4
:109CA00000000000000000000004000000040003A9
:109CB000000700030007E0010004F80100041F0290
:109CC000000007FC000000E000000700000438006E
:109CD0000007C000000600000004000000040000AF
:109CE0000000000000000000000000000000000074
:109CF0000000000000000000000000000000000064
:109D00000000000000000000000000000000000053
:109D10000000000000000000000000000000000043
:109D2000000000000000000000000000000780604C
:109D3000000600E0000403E0000407A000040E2079
:109D400000043C20000470200005E0200007802073
:109D500000070060000400E0000003800000000035
:109D600000000000000000000000000000000000F3
:109D700000000000000000000000000000000000E3
:109D800000000000000000000000000000000000D3
:109D900000000000000000000000000000000000C3
:109DA00000000000000000000000000000000000B3
:109DB00000000000000000000000000000000000A3
:109DC00000008000000080000001400007FE3FF816
:109DD0000800000410000002100000020000000053
:109DE0000000000000000000000000000000000073
:109DF0000000000000000000000000000000000063
:109E00000000000000000000000000000000000052
:109E10000000000000000000000000000000000042
:109E20000000000000000000000000000000000032
:109E30000000000000000000000000000000000022
:109E400000000000FFFFFFFF000000000000000016
:109E50000000000000000000000000000000000002
:109E600000000000000000000000000000000000F2
:109E700000000000000000000000000000000000E2
:109E800000000000000000000000000000000000D2
:109E900000000000000000000000000000000000C2
:109EA00000000000000000000000000010000002A0
:109EB000100000020800000407FE3FF80001400007
:109EC0000000800000008000000000000000000092
:109ED0000000000000000000000000000000000082
:109EE0000000000000000000000000000000000072
:109EF0000000000000000000000000000000000062
:109F00000000000000000000000000000000000051
:109F10000000000000000000000000000000000041
:109F200000000000000000001800000030000000E9
:109F30004000000040000000400000002000000041
:109F400030000000080000000400000002000000D3
:109F500002000000020000000C00000018000000D9
:109F600000000000000000000000000000000000F1
:109F700000000000000000000000000000000000E1
:109F800000000000000000000000000000000000D1
:109F900000000000000000000000000000000000C1
:109FA0000000000030313233343536373839414221
:109FB000434445464030580030313233343536372B
:0C9FC000383961626364656640307800E7
:040000050800029954
:00000001FF
